:100000000C94BB010C9495320C94C2320C94E30115
:100010000C94E3010C94E3010C94E3010C94E301D0
:100020000C94E3010C94E3010C94E3010C94CE06D0
:100030000C94E3010C94E3010C94E3010C94E301B0
:100040000C94A1310C94E3010C9444060C948006AA
:100050000C94E3010C94E3010C94E3010C94E30190
:100060000C94E3010C94E301084AD73B3BCE016EAC
:1000700084BCBFFDC12F3D6C74319ABD56833DDAFF
:100080003D00C77F11BED9E4BB4C3E916BAAAABE0E
:10009000000000803F05A84CCDB2D44EB93836A937
:1000A000020C50B9918688083CA6AAAA2ABE000074
:1000B00000803F0664EC1B3C04BC163E3BE5B93CAB
:1000C000C93C37C29E5A3D660498083EEA69AAAA0E
:1000D0003E000000803F2020BF0020BF00BF007C0A
:1000E0002020202020202020202020202020202010
:1000F00020202000C8202020202020202020202078
:1001000020C900C8202020202020202020202020BE
:10011000C97C00D820202020202020202020202042
:10012000D97C00C820202020202020202020202032
:10013000C97C00C820202020202020202020202032
:10014000C97C00207265766F00206172737369004C
:100150006D696E6F706F7364206C6962726570692F
:100160006C6F74002020202020BABBBCBDBE7C2058
:1001700020202020CACBCCCDCE7C00626F6F74696A
:100180006E672075703AEDF2F2F2F2F2F2F2F300DD
:1001900062617474657279207761726E696E67202E
:1001A0000074787069642076616C756573006261B3
:1001B000726F2074656D700074656D706469737022
:1001C00020006163746976652000706173736976DD
:1001D000650075617674616C6B2000736574757071
:1001E0002073637265656E7C7C7C0043686172205D
:1001F000446F6E650A00526561647920666F7220F3
:10020000466F6E740A0055706461746520436861BE
:10021000725365740000407A10F35A00A0724E18B1
:10022000090010A5D4E80000E87648170000E40BA8
:1002300054020000CA9A3B000000E1F5050000806E
:10024000969800000040420F000000A086010000C8
:1002500000102700000000E8030000000064000018
:100260000000000A00000000000100000000002C57
:1002700076D888DC674F0823DFC1DFAE59E1B1B71C
:1002800096E5E3E453C63AE651997696E8E6C284E9
:1002900026EB898C9B62ED407C6FFCEFBC9C9F4001
:1002A000F2BAA56FA5F490055A2AF75C936B6CF926
:1002B000676DC11BFCE0E40D47FEF520E6B500D0FC
:1002C000ED902E0300943577050080841E08000011
:1002D000204E0A000000C80C333333330F986E12DF
:1002E000831141EF8D2114893BE65516CFFEE6DBE5
:1002F00018D1844B381BF77C1D901DA4BBE424202F
:100300003284725E228100C9F124ECA1E53D276EA2
:10031000616E00696E660000000000240027002A5C
:100320000000000000250028002B00000000002332
:100330000026002900040404040404040402020248
:100340000202020303030303030102040810204016
:10035000800102040810200102040810200000009F
:100360000700020100000304060000000000000076
:1003700000004F04150811241FBECFEFD8E0DEBFE8
:10038000CDBF14E0A0E0B1E0ECE1F0E702C00590E1
:100390000D92AC30B107D9F716E0ACE0B4E001C083
:1003A0001D92AF3BB107E1F713E0C6E7D3E004C00D
:1003B0002297FE010E940838C237D107C9F70E9470
:1003C000D1330C940C380C940000FA01AA27283081
:1003D00051F1203181F1E8946F936E7F6E5F7F4F12
:1003E0008F4F9F4FAF4FB1E03ED0B4E03CD0670F8E
:1003F000781F891F9A1FA11D680F791F8A1F911DE1
:10040000A11D6A0F711D811D911DA11D20D009F430
:1004100068943F912AE0269F11243019305D319372
:10042000DEF6CF010895462F4770405D4193B3E05B
:100430000FD0C9F7F6CF462F4F70405D4A3318F002
:10044000495D31FD4052419302D0A9F7EACFB4E0B3
:10045000A6959795879577956795BA95C9F700976B
:100460006105710508959B01AC010A2E069457950C
:10047000479537952795BA95C9F7620F731F841F63
:10048000951FA01D0895283008F027E03327DA01D2
:10049000990F311D87FD916000966105710539F452
:1004A00032602E5F3D9330E32A95E1F708959F3F38
:1004B00030F080387105610509F03C5F3C5F3D9389
:1004C000913008F08068911DDF93CF931F930F93B5
:1004D000FF92EF92192F987F9695E92F9695969512
:1004E000E90FFF27E159FD4F99273327EE24FF2419
:1004F000A701E70105900894079428F4360FE71E3A
:10050000F81E491F511D660F771F881F991F0694FB
:10051000A1F70590079428F4E70EF81E491F561F0F
:10052000C11D770F881F991F661F0694A1F70590BC
:10053000079428F4F80E491F561FC71FD11D880FB6
:10054000991F661F771F0694A1F70590079420F462
:10055000490F561FC71FD81F990F661F771F881F87
:100560000694A9F784911095177041F0D695C79518
:1005700057954795F794E7941A95C1F7E5E1F2E0AE
:1005800068941590159135916591959105907FE24C
:100590007395E118F10A430B560BC90BD009C0F74C
:1005A000E10CF11E431F561FC91FD01D7EF470338E
:1005B00011F48A95E6CFE894015030F0080F0AF460
:1005C0000027021708F4202F2395022F7A3328F0F2
:1005D00079E37D932A95E9F710C07D932A9589F6F2
:1005E000069497956795379517951794E118F10A32
:1005F000430B560BC90BD00998F023957E91739548
:100600007A3308F070E37C932013B8F77E91706121
:100610007D9330F0839571E37D9370E32A95E1F744
:100620001124EF90FF900F911F91CF91DF919927A7
:1006300087FD90950895CF93DF93BC01823091059B
:1006400010F462E070E0A091BD06B091BE06ED012D
:1006500040E050E0E0E0F0E021C088819981861719
:10066000970769F48A819B81309719F0938382837D
:1006700004C09093BE068093BD06FE0134C0681787
:10068000790738F44115510519F08417950708F4D6
:10069000AC01FE018A819B819C01E9012097E9F66A
:1006A00041155105A9F1CA01861B970B049708F45F
:1006B000BA01E0E0F0E02AC08D919C911197841777
:1006C0009507F9F46417750781F412968D919C9142
:1006D0001397309719F09383828304C09093BE06DA
:1006E0008093BD06FD0132964CC0CA01861B970B54
:1006F000FD01E80FF91F6193719302978D939C930D
:1007000040C0FD01828193819C01D9011097A1F61F
:100710008091BB069091BC06892B41F48091AC027C
:100720009091AD029093BC068093BB064091AE02BF
:100730005091AF024115510541F44DB75EB780911C
:10074000AA029091AB02481B590B2091BB06309135
:10075000BC06CA01821B930B8617970780F0AB017A
:100760004E5F5F4F8417950750F0420F531F509311
:10077000BC064093BB06F9016193719302C0E0E0AF
:10078000F0E0CF01DF91CF910895CF93DF930097F1
:1007900009F450C0EC0122971B821A82A091BD0679
:1007A000B091BE06109709F140E050E0AC17BD07CC
:1007B00008F1BB83AA83FE0121913191E20FF31F5F
:1007C000AE17BF0779F48D919C911197280F391FAF
:1007D0002E5F3F4F3983288312968D919C911397FA
:1007E0009B838A834115510571F4D093BE06C09353
:1007F000BD0620C012968D919C911397AD01009774
:1008000011F0DC01D3CFFA01D383C283219131915E
:10081000E20FF31FCE17DF0769F488819981280F53
:10082000391F2E5F3F4FFA01318320838A819B81DC
:1008300093838283DF91CF910895FC0105906150ED
:1008400070400110D8F7809590958E0F9F1F0895E6
:10085000FC016150704001900110D8F7809590958F
:100860008E0F9F1F08956EBD0DB407FEFDCF8EB590
:1008700008958DE061E00E94EF328BE061E00E941C
:10088000EF328CE060E00E94EF328AE061E00E948B
:10089000EF321CBC80E58CBD8DB58EB508958CE023
:1008A00094E00E9439040895FC011382128288EEBC
:1008B00093E0A0E0B0E084839583A683B78381ECC6
:1008C00092E0918380830895FC018089803419F43B
:1008D00021E030E002C020E030E0C9010895FC01D1
:1008E000818990E00895FC01648745876687478782
:1008F000089580E090E0089580E090E0089580E021
:1009000090E008950895EF92FF921F93CF93DF93A5
:10091000162F7A0186E060E00E942E338CE094E08E
:1009200060E00E9433048CE094E060E00E943304B5
:100930008CE094E069E00E9433048CE094E0612F45
:100940000E943304C0E0D0E0F701EC0FFD1F1081DE
:100950008CE094E06AE00E9433048CE094E06C2F19
:100960000E9433048CE094E06BE00E9433048CE03E
:1009700094E0612F0E9433042196C633D10521F7FC
:100980008CE094E068E00E9433048CE094E060EA3C
:100990000E9433048CE094E060EA0E94330485FDF9
:1009A000F9CF8CE094E060E00E9433048CE094E0A6
:1009B0006CE00E94330486E061E00E942E33DF91F8
:1009C000CF911F91FF90EF9008951F93CF93DF93E6
:1009D000EC01162F86E060E00E942E338CE094E05C
:1009E00060E00E943304112319F0113059F404C05F
:1009F0008CE094E0688904C068896C618CE094E0C4
:100A00000E94330486E061E00E942E33DF91CF9193
:100A10001F910895EF92FF920F931F938EE1489FCD
:100A200070011124E60EF11C86E060E00E942E3376
:100A30000CE014E0C80165E00E943304C8016F2D8A
:100A40000E943304C80166E00E943304C8016E2D81
:100A50000E9433041F910F91FF90EF900895EF9241
:100A6000FF920F931F937C010CE014E0C80167E034
:100A70000E943304C8016FEF0E94330486E061E0F6
:100A80000E942E33F70187858F5F87871F910F9113
:100A9000FF90EF900895EF92FF920F931F93FC0148
:100AA000E7848EE1E89E700111248685E80EF11C32
:100AB00086E060E00E942E330CE014E0C80164E0A0
:100AC0000E943304C80163E00E943304C80165E05A
:100AD0000E943304C8016F2D0E943304C80166E0F0
:100AE0000E943304C8016E2D0E9433041F910F91A0
:100AF000FF90EF9008951F93CF93DF93EC01162F93
:100B00006C3731F40E942F05CE010E944B050AC0BC
:100B10008CE094E067E00E9433048CE094E0612F65
:100B20000E94330481E090E0DF91CF911F910895FE
:100B30000F931F9386E060E00E942E330CE014E0D8
:100B4000C80164E00E943304C80164E00E943304D9
:100B500086E061E00E942E331F910F9108951F934C
:100B6000CF93DF93EC01188A16E0198B8BEA96E09D
:100B700060E973E00E940131813049F480E4888BA0
:100B800088E0898B86E060E00E942E3302C0188ADC
:100B9000198B86E060E00E942E33DF91CF911F9188
:100BA00008950F931F93CF93DF93EC0186E061E0EC
:100BB0000E94EF3282E060E00E94EF3282E061E06A
:100BC0000E942E33CE010E94AF0586E060E00E94B5
:100BD0002E338CE094E06CEE0E9433048CE094E0C1
:100BE0006FEF0E943304182F8CE094E060E00E94C5
:100BF0003304688962608CE094E00E94330462E30D
:100C000070E080E090E00E94F7318CE094E06CE6C8
:100C10000E9433041F7E8CE094E0612F0E94330415
:100C20008889803419F00DE010E002C000E110E086
:100C300010920E0410920D0417C060910D04709173
:100C40000E04605F8CE094E00E9433048CE094E03A
:100C500069E00E94330480910D0490910E04019686
:100C600090930E0480930D0480910D0490910E04D6
:100C70008017910714F3CE0161E00E94E504DF9133
:100C8000CF911F910F9108951F920F920FB60F925F
:100C900011242F933F934F938F939F93EF93FF9341
:100CA0004091C60020919A0630919B062F5F3F4FDE
:100CB00080919E0690919F062823392380919C065F
:100CC00090919D062817390779F080919A069091A6
:100CD0009B06E091A006F091A106E80FF91F408362
:100CE00030939B0620939A06FF91EF919F918F91ED
:100CF0004F913F912F910F900FBE0F901F9018951D
:100D00001F920F920FB60F9211242F933F938F9340
:100D10009F93EF93FF932091A4063091A5068091B5
:100D2000A2069091A30628173907E9F08091A4063E
:100D30009091A506E091A806F091A906E80FF91F89
:100D400080818093C6008091A4069091A5060196AB
:100D50002091A6063091A706822393239093A5069F
:100D60008093A40610C02091A2063091A306809122
:100D7000A4069091A5062817390729F48091C1008F
:100D80008F7D8093C100FF91EF919F918F913F9153
:100D90002F910F900FBE0F901F9018951F920F92DA
:100DA0000FB60F9211248F939F938091CF0490914F
:100DB000D004892B51F08091D1049091D2040196F6
:100DC0009093D2048093D10409C08091D304909170
:100DD000D40401969093D4048093D3049F918F916F
:100DE0000F900FBE0F901F901895CF93DF93482F51
:100DF000EB0180913006833009F45DC0843028F423
:100E00008130C1F0823058F50AC0853009F4D2C073
:100E1000853008F4A8C0863009F0F2C0E9C04C3330
:100E200009F0EEC081E080933006488384EB809324
:100E30002F06E6C0842F90E0E0912F06F0E0E8272F
:100E4000F927E153FD4F208120932F06887F907072
:100E5000809741F582E080933006498329C0242F92
:100E600030E0E0912F06F0E0E227F327E153FD4F59
:100E7000808180932F0680912E068F5F80932E06AF
:100E8000823018F43B832A83BBC0922F88272A81A3
:100E90003B81820F931F9B838A830A978F3F910523
:100EA00021F018F010923006ABC083E0809330063A
:100EB00010922E06A5C0E42FF0E080912F0690E05E
:100EC000E827F927E153FD4F808180932F06609139
:100ED0002E066F5F60932E06623089F0633020F437
:100EE000613009F08DC006C0633091F0643009F0C4
:100EF00087C022C0842F90E0A0E0B0E018C0242F6B
:100F000030E040E050E0542F432F322F222707C01B
:100F1000242F30E040E050E0A901332722278C81C4
:100F20009D81AE81BF81820F931FA41FB51F8C834B
:100F30009D83AE83BF8364C0242F30E040E050E047
:100F4000522F4427332722278C819D81AE81BF8178
:100F5000820F931FA41FB51F8C839D83AE83BF8315
:100F600060933006A5CF242F30E0E0912F06F0E00B
:100F7000E227F327E153FD4F808180932F06809174
:100F80002E068F5F80932E06813019F08230C1F5D6
:100F900003C03987288734C0922F88272885398550
:100FA000280F391F398728878A819B810A97F1F09A
:100FB00085E07CCFE42FF0E080912F0690E0E827D9
:100FC000F927E153FD4F808180932F0620912E0653
:100FD0002F5F20932E0630E0FB01E20FF31F4187C5
:100FE0008A819B810A972817390750F086E05ECFE7
:100FF000C75FDE4F4883C950D14087E080933006F9
:1010000080913006873069F410923006C75FDE4F5A
:1010100090912F068881C950D140981711F48A8188
:1010200001C080E0DF91CF9108958F92AF92CF926F
:10103000EF92FF920F931F9385E994E060E045ECF7
:1010400050E024EC30E000EC10E0B1ECEB2EF12CA1
:10105000CC24C394A8E9AA2EF0E28F2E0E94712A14
:1010600082EB94E00E9454041092C5041092C604CE
:101070001092C7041092C8041092C9041092CA04B6
:101080001092CB041092CC041092CE041092CD0496
:101090001092C4041F910F91FF90EF90CF90AF90EA
:1010A0008F900895AF92BF92CF92DF92EF92FF920E
:1010B0000F931F93E0909606F09097060091980684
:1010C000109199068FE590E0A0E0B0E0E80EF91EDF
:1010D0000A1F1B1F0E94E9316E157F0580079107CB
:1010E00008F44EC0A090FA04B090FB04C090FC0439
:1010F000D090FD04C601B50120E030E040E85FE398
:101100000E947136181694F5E0904E06F0904F0646
:1011100000915006109151060E94E93120919606E7
:10112000309197064091980650919906621B730B77
:10113000840B950B0E9447359B01AC01C601B5019C
:101140000E947C3620E030E04AE754E40E94AE344E
:101150009B01AC01C801B7010E94E13360934E06C8
:1011600070934F0680935006909351060E94E93188
:1011700060939606709397068093980690939906CD
:101180001F910F91FF90EF90DF90CF90BF90AF90A5
:101190000895DF93CF9300D000D0CDB7DEB7FB0129
:1011A000E80FF91F628583859485258569838A8385
:1011B0009B832C83492F5C81782FCA010F900F905D
:1011C0000F900F90CF91DF910895AF92BF92DF9271
:1011D000EF92FF920F931F93CF93DF938C01809137
:1011E000310680FDE4C0F801F08085E994E06F2DC0
:1011F0000E94522BE801C75FDE4FEF2DF0E0E15374
:10120000FD4F80818883F801F18085E994E06F2D9E
:101210000E94522BEF2DF0E0888190E0E827F9271B
:10122000E153FD4F80818883F801F28085E994E0E5
:101230006F2D0E94522BEF2DF0E0888190E0E8277F
:10124000F927E153FD4F80818883F801F38085E918
:1012500094E06F2D0E94522BEF2DF0E0888190E0FA
:10126000E827F927E153FD4F80818883F801F48056
:1012700085E994E06F2D0E94522BEF2DF0E08881DC
:1012800090E0E827F927E153FD4F80818883F8013A
:101290002481358146815781232F342F452F5527AF
:1012A000F22E85E994E0622F0E94522BEF2DF0E0A0
:1012B000888190E0E827F927E153FD4F80818883FA
:1012C000F80124813581468157819A0144275527A9
:1012D000F22E85E994E0622F0E94522BEF2DF0E070
:1012E000888190E0E827F927E153FD4F80818883CA
:1012F000F8012481358146815781252F33274427E2
:101300005527F22E85E994E0622F0E94522BEF2D93
:10131000F0E0888190E0E827F927E153FD4F8081D4
:10132000888385E994E060E00E94522BE881F0E038
:10133000E153FD4F8081888385E994E060E00E945D
:10134000522BE881F0E0E153FD4F80818883F80162
:10135000828193810B9718F18AE0A82EB12CA00E00
:10136000B11E750112C0F701D1907F0185E994E0AB
:101370006D2D0E94522BED2DF0E0888190E0E82742
:10138000F927E153FD4F808188832E2D2A1930E003
:10139000F801828193810A972817390720F3075FA4
:1013A0001E4F85E994E0F80160810E94522BDF9185
:1013B000CF911F910F91FF90EF90DF90BF90AF9072
:1013C0000895DF93CF93CDB7DEB7CA50D1400FB6A3
:1013D000F894DEBF0FBECDBF2CE329836A832AE0D9
:1013E00030E03C832B83FC0184819581A681B78109
:1013F0008D839E83AF83B887CE0101960E94E50856
:10140000C65FDE4F0FB6F894DEBF0FBECDBFCF91E3
:10141000DF9108958BEA96E06AE773E00E9401315C
:10142000882331F586E696E6A6E6B0E48093330697
:1014300090933406A0933506B093360680E090E092
:10144000A0E8BFE38093370690933806A09339064F
:10145000B0933A0688EE93E090933C0680933B0667
:1014600081E880933D068DE880933E068DEF25C090
:1014700082E598EBAEE0B0E48093330690933406B7
:10148000A0933506B093360685E89BEEA1E5B0E45F
:101490008093370690933806A0933906B0933A06A6
:1014A00080EA94E190933C0680933B068BEF809317
:1014B0003D0686E680933E068AEF80933F060895B8
:1014C000FF920F931F930BEA16E0C8016CE773E0DD
:1014D0000E94013180937A06C8016EE773E00E9492
:1014E000013180937B06C80160E873E00E940131FE
:1014F00080935A06C8016EE873E00E940131809320
:101500007206C8016AE873E00E9401318093700698
:10151000C80164E873E00E94013180937C06C80131
:1015200066E873E00E94013180937D06C8016CE893
:1015300073E00E94013180936206C80162E973E0A2
:101540000E94013180937E06C80164E973E00E9425
:10155000013180936106C80164EF73E00E9401319C
:10156000F82EC80165EF73E00E940131382F20E0AA
:101570002F0D311D3093800620937F06C80166EF42
:1015800073E00E940131F82EC80167EF73E00E94FA
:101590000131382F20E02F0D311D3093820620932A
:1015A0008106C80168EF73E00E940131F82EC8017E
:1015B00069EF73E00E940131382F20E02F0D311DBB
:1015C0003093840620938306C8016BEF73E00E947A
:1015D0000131809359061F910F91FF900895BC012E
:1015E0008BEA96E00E94013108956091E4047091C5
:1015F000E5048091E6049091E70420E030E040E1CA
:1016000052E40E947C3620E030E044EB53E40E9438
:10161000AE340E94DF360E9416359B0125503040C3
:1016200037FF03C09B01215E3F4FA2E4B6E0F90102
:10163000E153FC4F80818C932F5F3F4F2432310563
:1016400014F020E030E0119686E0AD34B80779F769
:101650001C9208952F923F924F925F926F927F92C9
:101660008F929F92AF92BF92CF92DF92EF92FF92B2
:101670000F931F93DF93CF9300D000D000D0CDB74E
:10168000DEB7182F662E2091DA043091DB042A355C
:10169000310530F0C9018D549F4F89359105E8F42B
:1016A00037FF02C02D543F4FC90137FF03C090954B
:1016B00081959F4F8A3191053CF0F4E48F2E912C57
:1016C000E9ED2E2E312C1DC00A975CF17BE3872EAD
:1016D000912C62ED262E312C20C02B35310514F0D3
:1016E000235B3040C90137FF03C0909581959F4F20
:1016F0008A31910554F056E5852E912C4CED242E1F
:10170000312C37E0A32EB12C15C00A9754F02DE4EC
:10171000822E912C94ED292E312C88E0A82EB12C0C
:1017200009C005E0802E912CB8E32B2E312CA9E0C6
:10173000AA2EB12C6091DC047091DD04882777FD1E
:101740008095982F0E94493527EA32E94BE25CEBFD
:101750000E947C360E94503720E030E040EA50E49E
:101760000E947C3620E030E040E951E40E947C3663
:101770000E94DF3620E030E044E352E40E94E1338F
:101780000E941635712EFEEBCF2EFFEFDF2E9B0150
:10179000442737FD4095542F29833A834B835C833C
:1017A000E2EB4E2EE4E05E2E4AEF5FEF240E351E94
:1017B0006091DA047091DB04882777FD8095982F7B
:1017C0000E94493525E33AEF4EE85CE30E947C36FF
:1017D0000E9450377B018C01B601882777FD8095E8
:1017E000982F0E9449359B01AC01C801B7010E94A6
:1017F0007C367B018C0169817A818B819C810E947E
:1018000049359B01AC01C801B7010E94E1330E9438
:1018100016359B01CB0101978A35910508F071C0FF
:1018200062E170E00E94B6378B012F5F3F4FAEEE52
:10183000BFEF6A9FC0016B9F900D7A9F900D11249E
:10184000820F931F62E070E00E94B6376D837E8343
:10185000E62CE01A4E2D4C5F82EB94E0672D0E943F
:101860000A0500D000D000D0EDB7FEB73196ADB775
:10187000BEB712965C924E92119720E031E033830E
:1018800022838D819E81880D991D958384830E947A
:10189000502A4DB75EB74A5F5F4F0FB6F8945EBFF0
:1018A0000FBE4DBF8D819E818A159B0554F104307A
:1018B00011053CF593E0E90EC201672D4E2D0E9403
:1018C0000A0500D000D000D0EDB7FEB73196ADB715
:1018D000BEB712965C924E92119720E031E03383AE
:1018E00022834D815E81420D531D558344830E94A6
:1018F000502A8DB79EB706960FB6F8949EBF0FBEBE
:101900008DBFACE0B0E0CA0EDB1E7394BEE4CB1614
:10191000D10409F04DCF26960FB6F894DEBF0FBE66
:10192000CDBFCF91DF911F910F91FF90EF90DF908E
:10193000CF90BF90AF909F908F907F906F905F906F
:101940004F903F902F900895823010F422E002C013
:10195000282F220F30E08DB79EB708970FB6F89466
:101960009EBF0FBE8DBFEDB7FEB7319682EB94E000
:10197000ADB7BEB712969C938E93119783E091E01A
:101980009383828322573F4F358324832F5F3F4FBA
:10199000378326830E94502A8DB79EB708960FB6CC
:1019A000F8949EBF0FBE8DBF0895CF93DF93AC0117
:1019B000E091EC04F091ED04209140063091410655
:1019C000C9018C599F4F8E179F071CF4EA0121977C
:1019D00009C024563040E217F30714F0EA0102C0B0
:1019E000EA012196842F90E0C817D90729F08BEAE5
:1019F00096E04C2F0E940831CE01DF91CF910895DF
:101A00000F931F930BEA16E0C80163EF73E041E008
:101A10000E940831C80164EF73E043E10E9408317D
:101A2000C80165EF73E046E00E940831C80166EF27
:101A300073E040E10E940831C80167EF73E047E2BC
:101A40000E940831C80168EF73E048E80E9408313D
:101A5000C80169EF73E043E10E9408311F910F91C3
:101A60000895CF92DF92EF92FF920F931F937C0124
:101A7000D62EC72E02EB14E0C8016E2D4D2D0E940C
:101A80007304C8010E944B0500D000D0EDB7FEB72B
:101A90001283018383E391E0948383830E943F2A2E
:101AA000EDB7FEB71283018383E291E094838383D1
:101AB0000E943F2AEDB7FEB71283018383E191E0D4
:101AC000948383830E943F2AEDB7FEB7128301837C
:101AD00083E091E0948383830E943F2AEDB7FEB7B1
:101AE0001283018384EF90E0948383830E943F2AD2
:101AF0000F900F900F900F90C8010E942F05C70103
:101B000001966D2D7C2D0E942A0B1F910F91FF9045
:101B1000EF90DF90CF900895CF92DF92EF92FF92F7
:101B20000F931F93CF93DF93182F062F0E94E93155
:101B300028EE33E040E050E00E94C93769017A01A5
:101B4000C2EBD4E0CE01612F402F0E947304CE017E
:101B50000E944B058091080590910905892B09F495
:101B600053C000910A0510910B058DB79EB744979D
:101B70000FB6F8949EBF0FBE8DBFEDB7FEB731967E
:101B8000ADB7BEB71296DC93CE93119788E091E083
:101B90009383828383EB90E095838483C6016CE317
:101BA00070E00E94B637CB016CE370E00E94B6375C
:101BB000978386832AE330E031872087C6016CE370
:101BC00070E00E94B6379387828785E690E095871C
:101BD0008487C8016CE370E00E94A237CB016CE3FC
:101BE00070E00E94B63797878687318B208BC801BB
:101BF0006CE370E00E94A237938B828B0E94502A84
:101C00008DB79EB7449633C0ADB7BEB71C970FB61D
:101C1000F894BEBF0FBEADBFEDB7FEB731961296BA
:101C2000DC93CE93119780E291E09383828383EBE0
:101C300090E095838483C6016CE370E00E94B63720
:101C4000CB016CE370E00E94B637978386838AE30A
:101C500090E091878087C6016CE370E00E94B63700
:101C6000938782870E94502A8DB79EB70C960FB635
:101C7000F8949EBF0FBE8DBF82EB94E00E942F05AB
:101C8000DF91CF911F910F91FF90EF90DF90CF9058
:101C90000895EF92FF920F931F93282F462FA2EBE8
:101CA000EA2EA4E0FA2EC701622F0E947304C70136
:101CB0000E944B058DB79EB70A970FB6F8949EBF4A
:101CC0000FBE8DBF0DB71EB70F5F1F4FEDB7FEB72D
:101CD000F282E1828CE291E0F80193838283609149
:101CE0000C0570910D0580910E0590910F052091C6
:101CF0003706309138064091390650913A060E94D5
:101D00007C36F801648375838683978380EB90E04B
:101D1000918780870E94502A8DB79EB70A960FB68A
:101D2000F8949EBF0FBE8DBFC7010E942F051F9163
:101D30000F91FF90EF9008958F929F92AF92BF9274
:101D4000CF92DF92EF92FF920F931F93E82EF62E21
:101D500002EB14E0C8016E2D4F2D0E947304C801E0
:101D60000E944B058DB79EB70C970FB6F8949EBF97
:101D70000FBE8DBFEDB7FEB73196ADB7BEB71296A9
:101D80001C930E93119794E3892E91E0992E9382E0
:101D900082828DEEA82EB12CB582A4828091150589
:101DA00090911605A0911705B09118058683978329
:101DB000A087B187B3EFCB2ED12CD386C2860E94E9
:101DC000502A8DB79EB70C960FB6F8949EBF0FBEE3
:101DD0008DBFC8010E942F05F394C8016E2D4F2DB1
:101DE0000E947304C8010E944B05ADB7BEB71C9793
:101DF0000FB6F894BEBF0FBEADBFEDB7FEB73196BC
:101E000012961C930E93119793828282B582A482BC
:101E10008091190590911A05A0911B05B0911C05A0
:101E200086839783A087B187D386C2860E94502A73
:101E30008DB79EB70C960FB6F8949EBF0FBE8DBFA0
:101E4000C8010E942F05F394C8016E2D4F2D0E94EA
:101E50007304C8010E944B05ADB7BEB71C970FB6FF
:101E6000F894BEBF0FBEADBFEDB7FEB73196129668
:101E70001C930E93119793828282B582A4828091E3
:101E80001D0590911E05A0911F05B0912005868328
:101E90009783A087B187D386C2860E94502A8DB7C8
:101EA0009EB70C960FB6F8949EBF0FBE8DBFC801AB
:101EB0000E942F051F910F91FF90EF90DF90CF9020
:101EC000BF90AF909F908F9008950F931F93282FEE
:101ED000462F02EB14E0C801622F0E947304C80170
:101EE0000E944B058DB79EB70A970FB6F8949EBF18
:101EF0000FBE8DBFEDB7FEB73196ADB7BEB7129628
:101F00001C930E9311978EE391E09383828389EB68
:101F100090E09583848380910805909109059783CB
:101F2000868382E890E0918780870E94502A8DB74F
:101F30009EB70A960FB6F8949EBF0FBE8DBFC8011C
:101F40000E942F051F910F910895EF92FF920F931A
:101F50001F93282F462F32EBE32E34E0F32EC701D8
:101F6000622F0E947304C7010E944B058DB79EB774
:101F70000C970FB6F8949EBF0FBE8DBF0DB71EB75E
:101F80000F5F1F4FEDB7FEB7F282E18286E491E06A
:101F9000F8019383828384EE90E09583848360913B
:101FA000060570910705882777FD8095982F0E9478
:101FB00049352AE037ED43E25CE30E947C36F801C4
:101FC00066837783808791878FE890E09387828705
:101FD0000E94502A8DB79EB70C960FB6F8949EBFFC
:101FE0000FBE8DBFC7010E942F051F910F91FF905B
:101FF000EF9008950F931F93282F462F02EB14E0C4
:10200000C801622F0E947304C8010E944B058DB75E
:102010009EB70C970FB6F8949EBF0FBE8DBFEDB75D
:10202000FEB73196ADB7BEB712961C930E931197BB
:1020300086E491E09383828382EE90E095838483AB
:102040008091020590910305A0910405B0910505CA
:1020500086839783A087B1878EE890E093878287F5
:102060000E94502A8DB79EB70C960FB6F8949EBF6B
:102070000FBE8DBFC8010E942F051F910F910895BB
:102080000F931F93282F462F82EB94E0622F0E941C
:10209000730482EB94E00E944B058091E90488234D
:1020A00019F420E531E057C0813019F424E531E01E
:1020B00052C0823019F428E531E04DC0833019F464
:1020C0002CE531E048C0843019F420E631E043C00B
:1020D000853019F424E631E03EC0863019F428E654
:1020E00031E039C0873019F42CE631E034C0883053
:1020F00019F420E731E02FC0893019F424E731E0EA
:102100002AC08A3019F428E731E025C08B3019F451
:102110002CE731E020C08C3019F420E831E01BC0FE
:102120008D3019F424E831E016C08E3019F428E817
:1021300031E011C08F3019F42CE831E00CC080314F
:1021400019F420E931E007C0813119F024E931E0C8
:1021500002C025E931E08DB79EB708970FB6F89415
:102160009EBF0FBE8DBFEDB7FEB7319602EB14E0F8
:10217000ADB7BEB712961C930E93119789E991E003
:102180009383828380EE90E09583848337832683D4
:102190000E94502A8DB79EB708960FB6F8949EBF3E
:1021A0000FBE8DBFC8010E942F051F910F9108958A
:1021B0000F931F93282F462F02EB14E0C801622FC4
:1021C0000E947304C8010E944B058DB79EB70A9701
:1021D0000FB6F8949EBF0FBE8DBFEDB7FEB7319618
:1021E000ADB7BEB712961C930E9311978EE991E08E
:1021F0009383828387E890E0958384838091EA04C7
:102200009091EB049783868385E290E091878087A5
:102210000E94502A8DB79EB70A960FB6F8949EBFBB
:102220000FBE8DBFC8010E942F051F910F91089509
:102230000F931F93282F462F02EB14E0C801622F43
:102240000E947304C8010E944B058DB79EB70A9780
:102250000FB6F8949EBF0FBE8DBFEDB7FEB7319697
:10226000ADB7BEB712961C930E93119788EA91E012
:10227000938382838091DC049091DD049583848331
:1022800080EB90E09783868381EB90E09187808755
:102290000E94502A8DB79EB70A960FB6F8949EBF3B
:1022A0000FBE8DBFC8010E942F051F910F91089589
:1022B0000F931F93282F462F02EB14E0C801622FC3
:1022C0000E947304C8010E944B058DB79EB70A9700
:1022D0000FB6F8949EBF0FBE8DBFEDB7FEB7319617
:1022E000ADB7BEB712961C930E93119788EA91E092
:1022F000938382838091DA049091DB0495838483B5
:1023000080EB90E09783868382EB90E091878087D3
:102310000E94502A8DB79EB70A960FB6F8949EBFBA
:102320000FBE8DBFC8010E942F051F910F91089508
:102330000F931F93282F462F02EB14E0C801622F42
:102340000E947304C8010E944B058DB79EB70A977F
:102350000FB6F8949EBF0FBE8DBFEDB7FEB7319696
:10236000ADB7BEB712961C930E93119780EB91E018
:102370009383828381EE90E0958384838091B80279
:102380009091B9029783868385E290E09187808758
:102390000E94502A8DB79EB70A960FB6F8949EBF3A
:1023A0000FBE8DBFC8010E942F051F910F91089588
:1023B0000F931F93282F462F02EB14E0C801622FC2
:1023C0000E947304C8010E944B058DB79EB70C97FD
:1023D0000FB6F8949EBF0FBE8DBFEDB7FEB7319616
:1023E000ADB7BEB712961C930E93119788EB91E090
:1023F0009383828382EC91E09583848380ED90E0E7
:102400009783868382E496E09187808781ED90E0D0
:10241000938782870E94502A8DB79EB70C960FB67D
:10242000F8949EBF0FBE8DBFC8010E942F051F915B
:102430000F9108950F931F93282F462F02EB14E05E
:10244000C801622F0E947304C8010E944B058DB71A
:102450009EB70A970FB6F8949EBF0FBE8DBFEDB71B
:10246000FEB73196ADB7BEB712961C930E93119777
:1024700080ED91E0938382838091E4049091E50460
:10248000A091E604B091E70484839583A683B78383
:1024900080EB90E0918780870E94502A8DB79EB78D
:1024A0000A960FB6F8949EBF0FBE8DBFC8010E945A
:1024B0002F051F910F9108950F931F93282F462FDB
:1024C00002EB14E0C801622F0E947304C8010E944D
:1024D0004B058DB79EB70C970FB6F8949EBF0FBEF5
:1024E0008DBFEDB7FEB73196ADB7BEB712961C9350
:1024F0000E93119788ED91E09383828386E190E0BB
:10250000958384838091FE049091FF04A09100053F
:10251000B091010586839783A087B18788E890E012
:10252000938782870E94502A8DB79EB70C960FB66C
:10253000F8949EBF0FBE8DBFC8010E942F051F914A
:102540000F910895CF92DF92EF92FF920F931F9316
:10255000CF93DF93282F462FC2EBD4E0CE01622F1A
:102560000E947304CE010E944B0560914E0670914B
:102570004F06809150069091510620913706309178
:1025800038064091390650913A060E947C366B011C
:102590007C0120E030E04AE754E40E9471361816CE
:1025A000D4F58DB79EB70C970FB6F8949EBF0FBEAB
:1025B0008DBF0DB71EB70F5F1F4FADB7BEB71296D9
:1025C000DC93CE93119786E491E0F80193838283A4
:1025D0008EEF90E09583848360913B0670913C067A
:1025E000882777FD8095982F0E9449359B01AC0183
:1025F000C701B6010E94AE34D80116966D937D9343
:102600008D939C93199780913F061A968C931A97F5
:102610001B961C9221C08DB79EB70C970FB6F894ED
:102620009EBF0FBE8DBFEDB7FEB73196ADB7BEB73B
:102630001296DC93CE93119782EE91E0938382837E
:102640008EEF90E095838483C682D782E086F18600
:1026500080913E06828713860E94502AEDB7FEB70E
:102660003C960FB6F894FEBF0FBEEDBF82EB94E030
:102670000E942F05DF91CF911F910F91FF90EF9056
:10268000DF90CF900895EF92FF920F931F93282F22
:10269000462F52EBE52E54E0F52EC701622F0E9423
:1026A0007304C7010E944B058DB79EB70C970FB6F8
:1026B000F8949EBF0FBE8DBF0DB71EB70F5F1F4FA3
:1026C000EDB7FEB7F282E18288ED91E0F8019383E5
:1026D000828389EE90E0958384836091FA047091FF
:1026E000FB048091FC049091FD042091330630910D
:1026F000340640913506509136060E947C36F8012A
:10270000668377838087918780913D0682871386D1
:102710000E94502A8DB79EB70C960FB6F8949EBFB4
:102720000FBE8DBFC7010E942F051F910F91FF9013
:10273000EF900895EF92FF920F931F93282F462F4B
:1027400062EBE62E64E0F62EC701622F0E9473044E
:10275000C7010E944B058DB79EB70C970FB6F89432
:102760009EBF0FBE8DBF0DB71EB70F5F1F4FEDB7DA
:10277000FEB7F282E18282EE91E0F80193838283D8
:1027800086EE90E0958384836091F6047091F7045F
:102790008091F8049091F904209137063091380621
:1027A0004091390650913A060E947C36F8016683C2
:1027B00077838087918780913E06828713860E9467
:1027C000502A8DB79EB70C960FB6F8949EBF0FBED9
:1027D0008DBFC7010E942F051F910F91FF90EF90B1
:1027E0000895EF92FF920F931F93282F462F72EBBD
:1027F000E72E74E0F72EC701622F0E947304C70111
:102800000E944B058DB79EB70C970FB6F8949EBFEC
:102810000FBE8DBF0DB71EB70F5F1F4FEDB7FEB7D1
:10282000F282E18282EE91E0F8019383828387EE67
:1028300090E095838483609110057091110588273D
:1028400077FD8095982F0E94493520913706309169
:1028500038064091390650913A060E947C36F801BC
:10286000668377838087918780913E06828713866F
:102870000E94502A8DB79EB70C960FB6F8949EBF53
:102880000FBE8DBFC7010E942F051F910F91FF90B2
:10289000EF9008950F931F93282F462F02EB14E01B
:1028A000C801622F0E947304C8010E944B058091E9
:1028B00052060E94A40CC8010E942F051F910F917F
:1028C0000895EF92FF920F931F93282F462FE2EB6C
:1028D000EE2EE4E0FE2EC701622F0E947304C701B2
:1028E0000E944B058DB79EB70C970FB6F8949EBF0C
:1028F0000FBE8DBF0DB71EB70F5F1F4FEDB7FEB7F1
:10290000F282E18282EE91E0F801938382838FE18B
:1029100090E0958384836091530670915406809172
:102920005506909156060E94493520913706309100
:1029300038064091390650913A060E947C36F801DB
:10294000668377838087918780913E06828713868E
:102950000E94502A8DB79EB70C960FB6F8949EBF72
:102960000FBE8DBFC7010E942F051F910F91FF90D1
:10297000EF9008950F931F93282F462F02EB14E03A
:10298000C801622F0E947304C8010E944B058DB7D5
:102990009EB740970FB6F8949EBF0FBE8DBFEDB7A0
:1029A000FEB73196ADB7BEB712961C930E93119732
:1029B0008CEE91E09383828383E890E09583848317
:1029C0008091E0049091E104A091E204B091E304CD
:1029D00086839783A087B18784E890E09387828776
:1029E0008091F0049091F104A091F204B091F3046D
:1029F00084879587A687B7870E94502A8DB79EB790
:102A000040960FB6F8949EBF0FBE8DBFC8010E94BE
:102A10002F051F910F9108950F931F93282F462F75
:102A200082EB94E0622F0E94730482EB94E00E9498
:102A30004B058091F504282F30E0823030F4F4E02B
:102A4000220F331FFA95E1F702C02150304000D029
:102A500000D000D0EDB7FEB7319602EB14E0ADB771
:102A6000BEB712961C930E93119780E091E093836A
:102A70008283358324830E94502A8DB79EB70696A1
:102A80000FB6F8949EBF0FBE8DBFC8010E942F05E0
:102A90001F910F9108950F931F93282F462F02EB3C
:102AA00014E0C801622F0E947304C8010E944B0504
:102AB0008DB79EB708970FB6F8949EBF0FBE8DBF17
:102AC000EDB7FEB73196ADB7BEB712961C930E9315
:102AD00011978EEF91E0938382838FE090E095834E
:102AE00084838091F404868317820E94502A8DB7D4
:102AF0009EB708960FB6F8949EBF0FBE8DBFC80153
:102B00000E942F051F910F9108950F931F9302EBC1
:102B100014E0C80163E045E00E947304C8010E940C
:102B20004B0500D000D0EDB7FEB71283018384E6D9
:102B300091E0948383830E943F2AEDB7FEB712830E
:102B4000018380E591E0948383830E943F2AEDB75F
:102B5000FEB71283018389E491E0948383830E940A
:102B60003F2AEDB7FEB71283018383E491E094839B
:102B700083830E943F2A0F900F900F900F90C801FF
:102B80000E942F051F910F9108950F931F93282FD7
:102B9000462F02EB14E0C801622F0E947304C801A3
:102BA0000E944B0500D000D0EDB7FEB71283018321
:102BB0008BE791E0948383830E943F2A0F900F90CC
:102BC0000F900F90C8010E942F051F910F9108953B
:102BD000EF92FF920F931F93CF93DF930E94E931FF
:102BE00020915C0630915D0640915E0650915F0633
:102BF000261737074807590708F08AC10E94E931AC
:102C00006C507E4F8F4F9F4F60935C0670935D06B4
:102C100080935E0690935F0602EB14E0C8010E9469
:102C20009805C80165E043E00E947304C8010E9452
:102C30004B0500D000D0EDB7FEB7128301838BEDBA
:102C400091E0948383830E943F2A0F900F900F900E
:102C50000F908091400690914106892B31F0809130
:102C6000570690915806892B81F48091EC0490913D
:102C7000ED0490934106809340068091EE0490917C
:102C8000EF0490935806809357062091EE043091FC
:102C9000EF044091570650915806C9018456904060
:102CA0004817590724F480915B068F5F08C02C59A0
:102CB0003F4F241735072CF480915B068150809399
:102CC0005B0680915B06181614F081E003C0843027
:102CD0001CF083E080935B0680915B06823009F4F0
:102CE00062C0833009F4BEC0813009F00DC100D04C
:102CF00000D0C2EBD4E0EDB7FEB7D283C18382ED42
:102D000091E0948383830E943F2A809131060F9043
:102D10000F900F900F9080FF22C000D000D0EDB731
:102D2000FEB7D283C1838AEC91E0948383830E94AF
:102D30003F2A8091400690914106845690400F9022
:102D40000F900F900F902091EC043091ED04281714
:102D500039070CF0D9C0809131068E7F21C000D098
:102D600000D0EDB7FEB7D283C18382EC91E09483AB
:102D700083830E943F2A80914006909141068C599E
:102D80009F4F0F900F900F900F902091EC04309177
:102D9000ED04821793070CF0B7C080913106816073
:102DA00080933106B1C000D000D0C2EBD4E0EDB7C3
:102DB000FEB7D283C18388EB91E0948383830E9422
:102DC0003F2A0F900F900F900F9080915906882303
:102DD00001F100D000D0EDB7FEB7D283C1838EEAF7
:102DE00091E0948383830E943F2A809140069091D2
:102DF0004106845690400F900F900F900F902091B5
:102E0000EC043091ED04281739071CF5109259068F
:102E100020C000D000D0EDB7FEB7D283C18381EAD5
:102E200091E0948383830E943F2A80914006909191
:102E300041068C599F4F0F900F900F900F9020914B
:102E4000EC043091ED04821793071CF481E0809329
:102E500059068BEA96E06BEF73E0409159060E94A9
:102E6000083152C000D000D0A2EBEA2EA4E0FA2E26
:102E7000EDB7FEB7F282E18280E991E0948383832B
:102E80000E943F2A8DB79EB708970FB6F8949EBF51
:102E90000FBE8DBF0DB71EB70F5F1F4FEDB7FEB74B
:102EA000F282E18284E092E0F80193838283609170
:102EB0005A0670E080E090E00E94473520E030E064
:102EC00040E251E40E94AE34F80164837583868346
:102ED000978386E790E09187808780E290E09387F0
:102EE00082870E94502A8DB79EB70C960FB6F89431
:102EF0009EBF0FBE8DBF80915A0690E060E873E0E0
:102F00000E94D50C80935A0682EB94E00E942F0514
:102F1000DF91CF911F910F91FF90EF9008952F9225
:102F20003F924F925F926F927F928F929F92AF9259
:102F3000BF92CF92DF92EF92FF920F931F93DF9396
:102F4000CF93CDB7DEB72B970FB6F894DEBF0FBE89
:102F5000CDBF888769870E94E93120916906309149
:102F60006A0640916B0650916C0626173707480792
:102F7000590708F069C180916D068823C9F08093D4
:102F8000BA0210926D068CE092E090936F068093E7
:102F90006E060E94E9316C507E4F8F4F9F4F6093B9
:102FA000690670936A0680936B0690936C0607C15E
:102FB0008091BA02282E33242091E8042F830091B7
:102FC0006E0610916F063091D50439838091F50417
:102FD0008E83909160069D83E090220560900205AB
:102FE00070900305809004059090050590915A0615
:102FF0004090B8025090B90280916106A82FB0E0CD
:10300000BC83AB83B0916206BA83F09021053B8606
:103010002A86A92EBB24CC24DD24EA85FB853196A3
:10302000FB87EA8737972CF021E030E03B872A873F
:103030001CC08A859B858330910539F184309105C8
:103040003CF48130910589F0029709F07FC015C0EA
:10305000AA85BB85A530B10509F44EC0A530B105E0
:1030600004F1169709F072C058C0BF81B23008F061
:103070006DC009E112E081E070C0E981E33009F43C
:1030800065C006E212E082E068C0FE81F23008F01E
:103090005DC02D81222309F459C003E312E083E0CF
:1030A0005CC031E03E1598F0C601B5010E9447357D
:1030B00020E030E040E251E40E94AE349B01AC01DC
:1030C000C401B3010E94A73488230CF03FC000E480
:1030D00012E083E0E81649F094E0E91649F0A2E036
:1030E000EA1641F40DE412E005C00AE512E002C060
:1030F00007E612E084E031C0EB81FC814E165F06EA
:103100002CF5FDE94F16FFEF5F0601F12A8122231E
:10311000E9F404E712E085E020C03F813230B0F4EA
:1031200081E08F1598F493E0F91649F0A4E0FA16BF
:1031300049F0B2E0FB1651F401E812E005C00DE8D9
:1031400012E002C00AE912E086E007C0EA85FB85CA
:10315000E215F30509F061CF60C010936F0600938C
:103160006E0680936D0681E0809363060E94E931CC
:1031700068517C4F8F4F9F4F6093690670936A062A
:1031800080936B0690936C060E94E9316056704FF5
:103190008F4F9F4F60936506709366068093670616
:1031A0009093680680916406882321F082EB94E076
:1031B0000E9498051092640602C01092630602EB0A
:1031C00014E0C801688549850E947304C8010E9403
:1031D0004B0500D000D000D0EDB7FEB73196ADB7AB
:1031E000BEB712961C930E93119787EA92E09383D1
:1031F000828380916E0690916F06958384830E94EE
:10320000502AEDB7FEB736960FB6F894FEBF0FBE44
:10321000EDBFC8010E942F0517C010936F060093E1
:103220006E0610926D060E94E9312091650630917C
:1032300066064091670650916806261737074807CB
:10324000590708F4BACFBBCF2B960FB6F894DEBF60
:103250000FBECDBFCF91DF911F910F91FF90EF90E7
:10326000DF90CF90BF90AF909F908F907F906F90A6
:103270005F904F903F902F900895EF92FF920F93A1
:103280001F9380917006843009F056C09091E90434
:10329000943008F027C1809179068917A1F19093A5
:1032A00079060E94E93160937506709376068093E3
:1032B000770690937806909179068091BB029817D3
:1032C00011F580916406813091F0813018F08230E0
:1032D000B1F413C011E0109364060E94E931615308
:1032E00075478040904030F41093710608C082E02A
:1032F000809364061092710602C01092640682EBFD
:1033000094E00E9498050E94E93120917506309161
:1033100076064091770650917806621B730B840BFA
:10332000950B615D77408040904008F4DBC0809150
:10333000E9048093BB02D6C0853029F48091B002A5
:103340009091B10214C0863029F48091B20290911C
:10335000B3020DC0873029F48091B4029091B50278
:1033600006C0883041F48091B6029091B7029093E4
:1033700074068093730680917206209173063091D3
:103380007406882309F04AC0C901895097408F5AB2
:103390009440C8F40E94E9316153754780409040E1
:1033A00020F481E0809371060CC08091710688231F
:1033B00041F480916306882321F482EB94E00E941B
:1033C000980582E028C044E0203B340768F48091EF
:1033D0006406882349F01092710682EB94E00E9403
:1033E0009805109264067EC0205B34402955324017
:1033F00008F078C080916406813009F473C0809130
:103400006306882309F06EC01092710682EB94E087
:103410000E94980581E08093640664C0215B34407B
:1034200008F460C00E94E9316153754780409040C4
:1034300008F041C0809171068823E9F5E090750697
:10344000F0907606009177061091780688EE93E06A
:10345000A0E0B0E0E80EF91E0A1F1B1F0E94E93130
:10346000E616F70608071907E8F581E0809371066C
:1034700017C01092710682EB94E00E94980580912B
:103480006406823019F41092640603C08F5F809343
:10349000640680916406823018F082E080936406AE
:1034A0000E94E931609375067093760680937706E3
:1034B0009093780617C0E0907506F090760600911C
:1034C00077061091780688EE93E0A0E0B0E0E80E71
:1034D000F91E0A1F1B1F0E94E931E616F7060807AE
:1034E000190738F21F910F91FF90EF900895809186
:1034F0007006843010F00E943D1980917106882377
:1035000019F00E94E81508958091150480FF08C005
:1035100060917B048091790490E070E00E948F17A5
:1035200080916406823008F0FDC1A82FB0E0FD0153
:10353000E15FFB4F808185FF0BC0FD01E55DFB4F27
:103540006081A75DBB4F8C9190E070E00E944B15AD
:1035500080916406A82FB0E0FD01E15FFB4F808100
:1035600086FF0BC0FD01E15DFB4F6081A35DBB4F9A
:103570008C9190E070E00E940C1580916006882389
:1035800009F43FC080916406A82FB0E0FD01E15F1F
:10359000FB4F808187FF0BC0FD01ED5CFB4F60811D
:1035A000AF5CBB4F8C9190E070E00E94BA148091A8
:1035B0006406A82FB0E0FD01EF5EFB4F808184FF21
:1035C0000BC0FD01E55BFB4F6081A75BBB4F8C919E
:1035D00090E070E00E94611480916406A82FB0E032
:1035E000FD01EF5EFB4F808183FF0BC0FD01E95BB6
:1035F000FB4F6081AB5BBB4F8C9190E070E00E9411
:103600004A1480916406A82FB0E0FD01ED5EFB4FE7
:10361000808187FF0BC0FD01ED59FB4F6081AF59E1
:10362000BB4F8C9190E070E00E94F1138091640692
:10363000A82FB0E0FD01EB5EFB4F808183FF0BC044
:10364000FD01ED57FB4F6081AF57BB4F8C9190E070
:1036500070E00E945C1280916006882309F444C0E7
:103660008091F504823008F43FC080916406A82F51
:10367000B0E0FD01E95EFB4F808182FF0BC0FD01E0
:10368000E157FB4F6081A357BB4F8C9190E070E0F6
:103690000E94A21280916406A82FB0E0FD01ED5EA9
:1036A000FB4F808182FF0BC0FD01E15AFB4F60811F
:1036B000A35ABB4F8C9190E070E00E949A138091C6
:1036C0006406A82FB0E0FD01ED5EFB4F808183FF13
:1036D0000BC0FD01E959FB4F6081AB59BB4F8C9189
:1036E00090E070E00E94431380916406A82FB0E040
:1036F000FD01EF5EFB4F808181FF0BC0FD01E15CAE
:10370000FB4F6081A35CBB4F8C9190E070E00E9406
:103710001A1280916406A82FB0E0FD01EF5EFB4F06
:10372000808180FF0BC0FD01E55CFB4F6081A75CE1
:10373000BB4F8C9190E070E00E94D811809164069C
:10374000A82FB0E0FD01EB5EFB4F808186FF0BC030
:10375000FD01E557FB4F6081A757BB4F8C9190E06F
:1037600070E00E94981180916406A82FB0E0FD01DE
:10377000E15FFB4F808182FF0BC0FD01ED5DFB4FE0
:103780006081AF5DBB4F8C9190E070E00E9458115A
:1037900080916406A82FB0E0FD01E15FFB4F8081BE
:1037A00081FF0BC0FD01E15EFB4F6081A35EBB4F5B
:1037B0008C9190E070E00E94181180916406A82F0F
:1037C000B0E0FD01ED5EFB4F808184FF0BC0FD0189
:1037D000E159FB4F6081A359BB4F8C9190E070E0A1
:1037E0000E94D81080916406A82FB0E0FD01ED5E24
:1037F000FB4F808185FF0BC0FD01ED58FB4F6081C1
:10380000AF58BB4F8C9190E070E00E9440108091C7
:103810006406A82FB0E0FD01E15FFB4F808183FFCC
:103820000BC0FD01E95DFB4F6081AB5DBB4F8C912F
:1038300090E070E00E94FA0F80916406A82FB0E03B
:10384000FD01ED5EFB4F808180FF0BC0FD01E55A5D
:10385000FB4F6081A75ABB4F8C9190E070E00E94B3
:10386000A50F80916406A82FB0E0FD01E15FFB4F3A
:10387000808184FF0BC0FD01E95CFB4F6081AB5C84
:10388000BB4F8C9190E070E00E94650F80916406C0
:10389000A82FB0E0FD01E95EFB4F808181FF18C0D9
:1038A00080915906FD01EF56FB4F813049F4AD562A
:1038B000BB4F6C91808190E070E00E94490E08C07F
:1038C000AD56BB4F6C91808190E070E00E949C0EE1
:1038D00080916406A82FB0E0FD01EF5EFB4F808170
:1038E00087FF0BC0FD01E95AFB4F6081AB5ABB4F0C
:1038F0008C9190E070E00E948C0D80916406A82F5E
:10390000B0E0FD01ED5EFB4F808186FF0BC0FD0145
:10391000E958FB4F6081AB58BB4F8C9190E070E051
:103920000E94310D089582EB94E00E9498050E9458
:1039300085150E940A0A0895CF93DF93EC0182EB6C
:1039400094E00E946F04C817D9073CF082EB94E022
:103950000E946404892B09F42397CE01DF91CF9153
:103960000895EF92FF920F931F93CF93DF930091EF
:10397000640610E08AEF90E0089F7001099FF00C48
:10398000189FF00C1124C7010E94EF0AF801E15FB3
:10399000FB4F882319F08081816002C080818E7F77
:1039A000808380916406C82FD0E0C70102960E94F0
:1039B000EF0AC75EDB4F888380916406C82FD0E092
:1039C000C70104960E94EF0A90E00E949C1CC55E0D
:1039D000DB4F88830091640610E0C70188569F4F33
:1039E0000E94EF0AF801E15FFB4F882319F0808104
:1039F000806102C080818F7E808380916406C82FA1
:103A0000D0E0C70186569F4F0E94EF0ACB5CDB4F88
:103A1000888380916406C82FD0E0C70184569F4FE9
:103A20000E94EF0A90E00E949C1CC95CDB4F8883D7
:103A30000091640610E0C70106960E94EF0AF801A3
:103A4000E15FFB4F882319F08081826002C0808192
:103A50008D7F808380916406C82FD0E0C7010896CF
:103A60000E94EF0AC35EDB4F888380916406C82FF3
:103A7000D0E0C7010A960E94EF0A90E00E949C1CC9
:103A8000C15EDB4F88830091640610E0C7010C968D
:103A90000E94EF0AF801E15FFB4F882319F0808153
:103AA000846002C080818B7F808380916406C82FF0
:103AB000D0E0C7010E960E94EF0ACF5DDB4F8883EE
:103AC00080916406C82FD0E0C70140960E94EF0A9B
:103AD00090E00E949C1CCD5DDB4F888300916406C2
:103AE00010E0C70142960E94EF0AF801E15FFB4F28
:103AF000882319F08081886002C08081877F80835D
:103B000080916406C82FD0E0C70144960E94EF0A56
:103B1000CB5DDB4F888380916406C82FD0E0C7015E
:103B200046960E94EF0A90E00E949C1CC95DDB4F04
:103B300088830091640610E0C7014E960E94EF0A48
:103B4000F801E15FFB4F882319F08081806202C099
:103B500080818F7D808380916406C82FD0E0C7016B
:103B600080960E94EF0AC75DDB4F888380916406D0
:103B7000C82FD0E0C70182960E94EF0A90E00E9411
:103B80009C1CC55DDB4F88830091640610E0C70173
:103B900084960E94EF0AF801E15FFB4F882319F039
:103BA0008081806402C080818F7B808380916406E5
:103BB000C82FD0E0C70186960E94EF0AC35DDB4F95
:103BC000888380916406C82FD0E0C70188960E9440
:103BD000EF0A90E00E949C1CC15DDB4F888300913E
:103BE000640610E0C7018A960E94EF0AF801E15FBF
:103BF000FB4F882319F08081806802C080818F7715
:103C0000808380916406C82FD0E0C7018C960E9403
:103C1000EF0ACF5CDB4F888380916406C82FD0E029
:103C2000C7018E960E94EF0A90E00E949C1CCD5C1A
:103C3000DB4F88830091640610E0C701C0960E94A4
:103C4000EF0AF801EF5EFB4F882319F08081816055
:103C500002C080818E7F808380916406C82FD0E06F
:103C6000C701C2960E94EF0AC75CDB4F8883809130
:103C70006406C82FD0E0C701C4960E94EF0A90E006
:103C80000E949C1CC55CDB4F88830091640610E099
:103C9000C701C6960E94EF0AF801EF5EFB4F88232A
:103CA00019F08081826002C080818D7F8083809145
:103CB0006406C82FD0E0C701C8960E94EF0AC35C13
:103CC000DB4F888380916406C82FD0E0C701CA9675
:103CD0000E94EF0A90E00E949C1CC15CDB4F88832D
:103CE0000091640610E0C701CC960E94EF0AF8012B
:103CF000EF5EFB4F882319F08081846002C08081D1
:103D00008B7F808380916406C82FD0E0C701CE9658
:103D10000E94EF0ACF5BDB4F888380916406C82F37
:103D2000D0E0C701805C9F4F0E94EF0A90E00E94A4
:103D30009C1CCD5BDB4F88830091640610E0C701BB
:103D4000885B9F4F0E94EF0AF801EF5EFB4F8823CC
:103D500019F08081806102C080818F7E8083809194
:103D60006406C82FD0E0C701865B9F4F0E94EF0A10
:103D7000C75BDB4F888380916406C82FD0E0C70102
:103D8000845B9F4F0E94EF0A90E00E949C1CC55BE1
:103D9000DB4F88830091640610E0C7018E5B9F4F64
:103DA0000E94EF0AF801EF5EFB4F882319F0808133
:103DB000886002C08081877F808380916406C82FDD
:103DC000D0E0C7018C5B9F4F0E94EF0ACB5BDB4FBB
:103DD000888380916406C82FD0E0C7018A5B9F4F1B
:103DE0000E94EF0A90E00E949C1CC95BDB4F888315
:103DF0000091640610E0C701805B9F4F0E94EF0AAC
:103E0000F801EF5EFB4F882319F08081806202C0C9
:103E100080818F7D808380916406C82FD0E0C701A8
:103E20008E5A9F4F0E94EF0AC35BDB4F88838091BD
:103E30006406C82FD0E0C7018C5A9F4F0E94EF0A3A
:103E400090E00E949C1CC15BDB4F8883009164065C
:103E500010E0C7018A5A9F4F0E94EF0AF801EF5EF7
:103E6000FB4F882319F08081806402C080818F7BA2
:103E7000808380916406C82FD0E0C701885A9F4F85
:103E80000E94EF0ACF5ADB4F888380916406C82FC7
:103E9000D0E0C701865A9F4F0E94EF0A90E00E942F
:103EA0009C1CCD5ADB4F88830091640610E0C7014B
:103EB00082569F4F0E94EF0AF801EF5EFB4F882366
:103EC00019F08081806802C080818F778083809123
:103ED0006406C82FD0E0C70180569F4F0E94EF0AAA
:103EE000CB5ADB4F888380916406C82FD0E0C7018E
:103EF0008E559F4F0E94EF0A90E00E949C1CC95A69
:103F0000DB4F88830091640610E0C7018E599F4FF4
:103F10000E94EF0AF801ED5EFB4F882319F08081C3
:103F2000816002C080818E7F808380916406C82F6B
:103F3000D0E0C7018C599F4F0E94EF0AC75ADB4F50
:103F4000888380916406C82FD0E0C7018A599F4FAB
:103F50000E94EF0A90E00E949C1CC55ADB4F8883A8
:103F60000091640610E0C70182599F4F0E94EF0A3A
:103F7000F801ED5EFB4F882319F08081846002C058
:103F800080818B7F808380916406C82FD0E0C70139
:103F900080599F4F0E94EF0AC35ADB4F888380915C
:103FA0006406C82FD0E0C7018E589F4F0E94EF0AC9
:103FB00090E00E949C1CC15ADB4F888300916406EC
:103FC00010E0C70184579F4F0E94EF0AF801ED5E91
:103FD000FB4F882319F08081806802C080818F7731
:103FE000808380916406C82FD0E0C70182579F4F1D
:103FF0000E94EF0ACF59DB4F888380916406C82F57
:10400000D0E0C70180579F4F0E94EF0A90E00E94C6
:104010009C1CCD59DB4F88830091640610E0C701DA
:104020008E569F4F0E94EF0AF801ED5EFB4F8823EA
:1040300019F08081826002C080818D7F80838091B1
:104040006406C82FD0E0C7018C569F4F0E94EF0A2C
:10405000C759DB4F888380916406C82FD0E0C70121
:104060008A569F4F0E94EF0A90E00E949C1CC559FF
:10407000DB4F88830091640610E0C7018C589F4F86
:104080000E94EF0AF801ED5EFB4F882319F0808152
:10409000886002C08081877F808380916406C82FFA
:1040A000D0E0C7018A589F4F0E94EF0ACB59DB4FDF
:1040B000888380916406C82FD0E0C70188589F4F3D
:1040C0000E94EF0A90E00E949C1CC959DB4F888334
:1040D0000091640610E0C70186589F4F0E94EF0AC6
:1040E000F801ED5EFB4F882319F08081806102C0EA
:1040F00080818F7E808380916406C82FD0E0C701C5
:1041000084589F4F0E94EF0AC359DB4F88838091E8
:104110006406C82FD0E0C70182589F4F0E94EF0A63
:1041200090E00E949C1CC159DB4F8883009164067B
:1041300010E0C70180589F4F0E94EF0AF801ED5E22
:10414000FB4F882319F08081806202C080818F7DBF
:10415000808380916406C82FD0E0C7018E579F4F9F
:104160000E94EF0ACF58DB4F888380916406C82FE6
:10417000D0E0C7018C579F4F0E94EF0A90E00E9449
:104180009C1CCD58DB4F88830091640610E0C7016A
:104190008A579F4F0E94EF0AF801ED5EFB4F88237C
:1041A00019F08081806402C080818F7B8083809140
:1041B0006406C82FD0E0C70188579F4F0E94EF0ABE
:1041C000CB58DB4F888380916406C82FD0E0C701AD
:1041D00086579F4F0E94EF0A90E00E949C1CC9588E
:1041E000DB4F88830091640610E0C7018C559F4F18
:1041F0000E94EF0AF801EB5EFB4F882319F08081E3
:10420000816002C080818E7F808380916406C82F88
:10421000D0E0C7018A559F4F0E94EF0AC758DB4F75
:10422000888380916406C82FD0E0C70188559F4FCE
:104230000E94EF0A90E00E949C1CC558DB4F8883C7
:104240000091640610E0C70180559F4F0E94EF0A5D
:10425000F801EB5EFB4F882319F08081846002C077
:1042600080818B7F808380916406C82FD0E0C70156
:104270008E549F4F0E94EF0AC358DB4F8883809172
:104280006406C82FD0E0C7018C549F4F0E94EF0AEC
:1042900090E00E949C1CC158DB4F8883009164060B
:1042A00010E0C7018A549F4F0E94EF0AF801EB5EAD
:1042B000FB4F882319F08081886002C08081877F4E
:1042C000808380916406C82FD0E0C70188549F4F37
:1042D0000E94EF0ACF57DB4F888380916406C82F76
:1042E000D0E0C70186549F4F0E94EF0A90E00E94E1
:1042F0009C1CCD57DB4F88830091640610E0C701FA
:1043000084549F4F0E94EF0AF801EB5EFB4F882315
:1043100019F08081806102C080818F7E80838091CE
:104320006406C82FD0E0C70182549F4F0E94EF0A55
:10433000CB57DB4F888380916406C82FD0E0C7013C
:1043400080549F4F0E94EF0A90E00E949C1CC95726
:10435000DB4F88830091640610E0C701845A9F4FA9
:104360000E94EF0AF801EB5EFB4F882319F0808171
:10437000806402C080818F7B808380916406C82F17
:10438000D0E0C701825A9F4F0E94EF0AC757DB4F08
:10439000888380916406C82FD0E0C701805A9F4F60
:1043A0000E94EF0A90E00E949C1CC557DB4F888357
:1043B0000091640610E0C70180529F4F0E94EF0AEF
:1043C000F801E95EFB4F882319F08081846002C008
:1043D00080818B7F808380916406C82FD0E0C701E5
:1043E0008E519F4F0E94EF0AC357DB4F8883809105
:1043F0006406C82FD0E0C7018C519F4F0E94EF0A7E
:1044000090E00E949C1CC157DB4F8883009164069A
:1044100010E0C7018C529F4F0E94EF0AF801E95E3D
:10442000FB4F882319F08081826002C080818D7FDC
:10443000808380916406C82FD0E0C7018A529F4FC5
:104440000E94EF0ACF56DB4F888380916406C82F05
:10445000D0E0C70188529F4F0E94EF0A90E00E946F
:104460009C1CCD56DB4F8883DF91CF911F910F911C
:10447000FF90EF9008954F925F927F928F929F925C
:10448000AF92BF92CF92DF92EF92FF920F931F9362
:10449000DF93CF93CDB7DEB7C854D0400FB6F894B2
:1044A000DEBF0FBECDBF02EB14E0C8010E9498052D
:1044B000C80166E049E00E947304C8010E944B05F0
:1044C00000D000D0EDB7FEB71283018386E092E002
:1044D000948383830E943F2A0F900F900F900F9038
:1044E000C8010E942F0500D000D005E914E0EDB707
:1044F000FEB71283018386EF91E0948383830E9449
:104500003F2A4BEE442E41E0542EEE24FF24CC24CF
:10451000DD240F900F900F900F90702E012F39E037
:10452000A32EB12CAC0EBD1E4E010894811C911C13
:1045300085E994E00E94F32A982F8D3031F08D3078
:10454000DCF180538230C0F530C01830A1F599817C
:10455000892F8053823078F5913311F490E801C0AF
:1045600090E08A81813309F4905C8B81813309F476
:10457000905E8C81813309F4905F8D81813309F4E1
:10458000985F8E81813309F49C5F8F81813309F4B8
:104590009E5F8885813309F49F5FF501EE0DFF1D55
:1045A00090830894E11CF11C06C0F401E10FF11D99
:1045B00090831F5F01C010E0F0E4EF16F104C9F42E
:1045C00082EB94E0B601A5010E9483040894C11C0B
:1045D000D11C00D000D0EDB7FEB7718202835482A7
:1045E00043820E943F2AEE24FF240F900F900F90E9
:1045F0000F90FFEFCF16D10409F00CF499CFC85BF0
:10460000DF4F0FB6F894DEBF0FBECDBFCF91DF9165
:104610001F910F91FF90EF90DF90CF90BF90AF90E0
:104620009F908F907F905F904F900895DF92EF92D0
:10463000FF920F931F93DF93CF93CDB7DEB72A97E7
:104640000FB6F894DEBF0FBECDBF63E0E62EF12CAF
:10465000EC0EFD1E53E0D52EF6C30E94E9316052E8
:104660007E4480409040C8F40E94E931695873410B
:104670008040904090F01A3011F01D3031F480915C
:104680002D068F5F80932D0602C010922D0680911B
:104690002D06833011F40E943B22812F63E275E0E6
:1046A0000E94F506882311F400E0C7C38091270516
:1046B00090912805A0912905B0912A05863E46EAE9
:1046C000940746E2A4074DE7B40709F48EC2873E7B
:1046D00056EA950756E2A5075DE7B50708F0EFC073
:1046E0008832EEE59E07E2EDAE07E4E2BE0709F48C
:1046F00027C28932FEE59F07F2EDAF07F4E2BF075C
:1047000008F06AC088392CE292072AE1A20726E164
:10471000B20709F41EC289393CE293073AE1A307C4
:1047200036E1B30740F586314AEA940747E3A40728
:104730004BE0B40709F404C287315AEA950757E3FE
:10474000A5075BE0B50738F48E5F9B4CA74CB940DA
:1047500009F069C360C38430FAE99F07F7EDAF073A
:10476000FEE0BF0709F4ECC18259934AAC4EB44154
:1047700009F059C3E5C184373BEE93073AE7A30735
:104780003BE1B30709F4DCC185374BEE94074AE7F8
:10479000A4074BE1B40780F480355FED95075DEE2B
:1047A000A50758E1B50709F40BC38E5C9844A745EB
:1047B000BA4109F038C319C28434FBED9F07F0E712
:1047C000AF07FDE1BF0709F426C3825D924CA24802
:1047D000BE4109F028C3BDC1883536EB93073DEFD4
:1047E000A3073AE4B30709F4CDC2893546EB940731
:1047F0004DEFA4074AE4B40788F5863E55ED9507CA
:104800005AEDA50753E3B50709F448C1873EE5ED26
:104810009E07EAEDAE07E3E3BE0780F48E37F9EAC0
:104820009F07FBE5AF07F6E2BF0709F492C1825587
:104830009342A649B64209F0F6C254C2883F3CEA08
:1048400093073EEEA30734E3B30709F4E4C2865AA4
:104850009E40A241B84409F0E6C27DC280365BEDBD
:1048600095075BE3A5075EE6B50709F469C18136E4
:10487000EBED9E07EBE3AE07EEE6BE0780F4823E6B
:10488000F5E59F07FCE9AF07F6E6BF0709F48AC222
:104890008C5E9943A647BB4609F0C5C2BCC28A3BA1
:1048A00037EC930731E2A30734E7B30709F4F6C006
:1048B0008A57974CA94DBB4709F0B5C2ACC28A3B99
:1048C00054E8950755E2A5075EEBB50709F46AC2FF
:1048D0008B3BE4E89E07E5E2AE07EEEBBE0708F08F
:1048E0006AC08E37F2E19F07FAE6AF07FBE9BF0720
:1048F00009F426C18F3722E192072AE6A2072BE9A5
:10490000B20740F582353AEE930730E8A3073AE85C
:10491000B30709F415C183354AEE940740E8A407AC
:104920004AE8B40738F486549340A24CB54809F0DD
:104930007AC271C28C38E5E89E07E7EAAE07E8E97B
:10494000BE0709F452C18A569E42A246B94909F0EF
:104950006AC201C280322EE4920729EAA20721EB43
:10496000B20709F41FC281323EE4930739EAA30774
:1049700031EBB30780F48A3746EF940741EFA40781
:104980004DE9B40709F431C18E5F964BA942B54A8F
:1049900009F049C22AC18A38E7EF9E07E7ECAE0763
:1049A000E8EBBE0709F4D5C0845A9040AB49BA4B36
:1049B00009F039C230C2843629ED920720EEA207F1
:1049C00027EDB20709F46AC0853639ED930730EE5A
:1049D000A30737EDB30788F586384BE3940740EA21
:1049E000A40744ECB40709F4DDC187385BE39507FD
:1049F00050EAA50754ECB50780F48C36E8E69E072C
:104A0000E3E4AE07E2ECBE0709F45CC180589447CA
:104A1000A041B44C09F007C29CC084352DE2920736
:104A20002FEFA20725ECB20709F48AC086599543F7
:104A3000A840B24D09F0F7C155C18E344DE5940739
:104A40004EE3A40743EEB40709F47AC08F345DE562
:104A500095075EE3A50753EEB50780F48437E7E3D7
:104A60009E07E4EDAE07EEEDBE0709F49BC1865B41
:104A70009342A34AB24E09F0D6C1B7C0823920E7AB
:104A8000920726E8A2072BEFB20709F4C4C1825FA0
:104A90009D4EA442BD4F09F0C6C18DC10E94E931AF
:104AA0006093D6047093D7048093D8049093D9046C
:104AB000D092D50483E295E060E170E00E94C908DD
:104AC0000E9416357093DB046093DA0483E295E06C
:104AD00064E170E00E94C9080E9416357093DD04FD
:104AE0006093DC0483E295E068E170E00E94C9080D
:104AF0000E9416358B017093DF046093DE04609191
:104B0000E0047091E1048091E2049091E30420E0DC
:104B100030E040E050E00E94A734882379F4B801E7
:104B2000882777FD8095982F0E9449356093E4048B
:104B30007093E5048093E6049093E70401E074C168
:104B400080912D058093E80480912E058093E904DF
:104B50006AC183E295E060E070E00E94C90820E04D
:104B600030E048EC52E40E947C360E941635709387
:104B7000EB046093EA04693C710520F01092EB04A9
:104B80001092EA0480914705909148059093ED04B6
:104B90008093EC048091490590914A059093EF042D
:104BA0008093EE0480914D0590914E059093B10253
:104BB0008093B00280915105909152059093B30279
:104BC0008093B20280915305909154059093B50261
:104BD0008093B40280915505909156059A838983FC
:104BE0009093B7028093B6021EC160912D0570911B
:104BF0002E0580912F05909130050E94493520E8BF
:104C000036E948E15BE40E94AE346093E0047093BF
:104C1000E1048093E2049093E30460913105709184
:104C200032058091330590913405D7016C9311962C
:104C30007C93119712968C93129713969C930E94D3
:104C4000493520E836E948E15BE40E94AE346093E0
:104C5000F0047093F1048093F2049093F304809134
:104C600052058093F404809151058093F50483E20A
:104C700095E060E170E00E94C9086093E4047093DD
:104C8000E5048093E6049093E70483E295E068E00E
:104C900070E00E94C9086093F6047093F704809353
:104CA000F8049093F90483E295E064E170E00E94D7
:104CB000C9086093FA047093FB048093FC049093FA
:104CC000FD04B1C083E295E068E070E00E94C9088D
:104CD00090586093FE047093FF04809300059093B6
:104CE0000105A1C083E295E060E070E00E94C90880
:104CF0006093020570930305809304059093050566
:104D000083E295E064E070E00E94C90820E030E0B2
:104D100048EC52E40E947C360E94163570930705D9
:104D20006093060583E295E064E170E00E94C908A3
:104D30000E941635709309056093080583E295E09B
:104D400068E170E00E94C9080E94163570930B0557
:104D500060930A0568C083E295E064E070E00E9419
:104D6000C9080E941635882777FD8095982F0E94E4
:104D7000493560930C0570930D0580930E05909353
:104D80000F0551C083E295E068E070E00E94C90819
:104D90000E941635709561957F4F70931105609351
:104DA000100541C080918D058093120580918E057C
:104DB0008093130538C080912D058093140533C06E
:104DC00083E295E060E070E00E94C90860931505F9
:104DD00070931605809317059093180583E295E06C
:104DE00064E070E00E94C9086093190570931A0589
:104DF00080931B0590931C0583E295E068E070E0CA
:104E00000E94C90860931D0570931E0580931F05BD
:104E10009093200508C080913905809321058091E9
:104E20003E058093220500E080912405823229F41A
:104E300083E295E063E20E94E1098EEB90E00E943C
:104E40005032002331F585E994E00E94C32A1816F8
:104E50001906F4F485E994E00E94F32A182F809152
:104E6000D504882309F019CCF8CB1092D50401E0C1
:104E7000802F90E02A960FB6F894DEBF0FBECDBF0C
:104E8000CF91DF911F910F91FF90EF90DF900895E8
:104E900000E02091D6043091D7044091D80450917D
:104EA000D904205F384D4F4F5F4F2F833887498794
:104EB0005A870E94E9312F81388549855A852617FE
:104EC00037074807590788F2D3CFEF92FF920F9325
:104ED0001F9380916206882351F083E00E948533FE
:104EE00064E070E00E94B637609332063CC083E015
:104EF0000E948533AA2797FDA095BA2FBC01CD014A
:104F00000E9449352DEC3CEC4CE45EE30E947C367B
:104F100020E030E040E85EE30E947C367B018C01BB
:104F20006091320670E0882777FD8095982F0E9467
:104F300049352DEC3CEC4CE45FE30E947C369B0150
:104F4000AC01C801B7010E94E1330E941B352091DA
:104F50007D06621730F030917C06262F361708F454
:104F6000232F209332061F910F91FF90EF90089509
:104F700083E00E94823308951F93CF93DF9385E0EF
:104F800090E06CE070E00E94C51568EE73E080E090
:104F900090E00E94F73185E994E00E94402BC0E048
:104FA000D0E010E0CE016DE171E00E94B637892BB0
:104FB000A9F41F5E82EB94E0612F4CE00E94730421
:104FC00082EB94E00E944B0582EB94E06EEE0E942F
:104FD0007B0582EB94E00E942F05105161E070E0A8
:104FE00080E090E00E94F731219687E0C13DD8072C
:104FF000C9F6DF91CF911F91089586E061E00E948C
:105000002E3308950F931F9386E061E00E94EF32E4
:1050100005E914E0C80140E051EE60E070E00E9454
:10502000612A1093AD060093AC060E94FD2782EB27
:1050300094E00E94D1050E94931C64EF71E080E02F
:1050400090E00E94F73183EF93E00E94EF0A8130F5
:1050500011F00E94000D0E94600A1092640607C0C1
:105060000E94B11C809164068F5F809364068091DA
:1050700064068230A8F3109264060E94BC270E9446
:10508000B82784EC94E063ED79E224E630E040E078
:1050900050E000E00E94143182EB94E00E949805F9
:1050A00084EC94E00E947A311F910F9108952F9221
:1050B0003F924F925F926F927F928F929F92AF92A8
:1050C000BF92CF92DF92EF92FF920F931F93DF93E5
:1050D000CF9300D000D0CDB7DEB780916006882393
:1050E00009F4E1C0E0908506F090860600918706FD
:1050F00010918806C801B7019F7725E33AEF4EE883
:105100005CE30E947C360E94AB3469837A838B8394
:105110009C83C801B7012091E0043091E1044091E3
:10512000E2045091E3040E94E0331B012C019F77BD
:1051300020EC3BE649ED57E40E947C365B016C01B4
:105140006091890670918A0680918B0690918C06F9
:105150002091F0043091F1044091F2045091F30455
:105160000E94E0333B014C019F7720EC3BE649ED88
:1051700057E40E947C3629813A814B815C810E94F0
:105180007C367B018C01C601B501A60195010E9408
:105190007C365B016C01C801B701A80197010E9430
:1051A0007C369B01AC01C601B5010E94E1330E942F
:1051B00003370E941635609353067093540680930C
:1051C00055069093560660E070E080E89FE32981E1
:1051D0003A814B815C810E94AE349B01AC01C201DB
:1051E000B1010E947C3697FA909497F89094A401AC
:1051F00093010E94543420EE3EE245E652E40E94C0
:105200007C3620E030E044EB52E40E94E1330E941F
:1052100016359B01AC0197FF04C028593E4F4F4FF4
:105220005F4FCA01B901645B70408040904097FFB6
:1052300006C0CA01B9016C547F4F8F4F9F4F0E9427
:1052400049352091E4043091E5044091E604509101
:10525000E7040E94E0330E94163597FF04C06859A6
:105260007E4F8F4F9F4F0E94493520E030E044EB46
:1052700053E40E94AE3420E030E040E851E40E9464
:105280007C360E94DF3620E030E040E85FE30E9499
:10529000E1330E941B3560935206613108F46CC003
:1052A0001092520669C08091F504823008F464C0FF
:1052B0008091F404853008F45FC0A0908D068DE1E4
:1052C0008A1508F459C0E090F604F090F7040091B4
:1052D000F8041091F90460918E0670918F06809108
:1052E000900690919106A80197010E94E0339F7764
:1052F00020E030E040E05FE30E94713618165CF475
:1053000010928D06E0928E06F0928F060093900622
:105310001093910631C08A2D8F5F80938D068E3158
:1053200059F58091E0049091E104A091E204B091DC
:10533000E3048093850690938606A0938706B09336
:1053400088068091F0049091F104A091F204B0914C
:10535000F3048093890690938A06A0938B06B093FA
:105360008C06E0929206F0929306009394061093B6
:10537000950681E0809360060F900F900F900F903C
:10538000CF91DF911F910F91FF90EF90DF90CF9021
:10539000BF90AF909F908F907F906F905F904F9055
:1053A0003F902F900895CF92DF92EF92FF920F934C
:1053B0001F930E94652780913206282F30E030939A
:1053C000B9022093B80280916206882359F50091B2
:1053D0007D0610E0201B310BB901882777FD8095F1
:1053E000982F0E9449356B017C0160917C0670E02A
:1053F000601B710B882777FD8095982F0E94493597
:105400009B01AC01C701B6010E94AE3420E030E040
:1054100048EC52E40E947C360E9416357093B90223
:105420006093B8028091B8029091B9028D599F4F54
:1054300034F48DE99FEF9093B9028093B8020E94F3
:1054400052080E94F50A82EB94E00E9457280E94BD
:10545000771A1F910F91FF90EF90DF90CF900895F2
:105460000E941623892B19F00E94D329089584ECF9
:1054700094E00E94623108958FEF9FE70895DF93D3
:10548000CF93CDB7DEB7FE0139968D819E8161E065
:105490004F8158859F010E94E02CCF91DF910895A4
:1054A000DF93CF93CDB7DEB7FE0139968D819E8114
:1054B00060E04F8158859F010E94E02CCF91DF91E1
:1054C00008950F931F93DC01ED91FC910288F389FD
:1054D000E02D20E030E000E010E009951F910F91F1
:1054E00008958F92AF92CF92EF92FF920F931F93F6
:1054F000DF93CF93CDB7DEB7FC011382128288EE23
:1055000093E0A0E0B0E084839583A683B78387EF20
:1055100093E0918380835587448737872687118B53
:10552000008BF38AE28AC48AA58A868A70E0CB015E
:1055300023E0880F991F2A95E1F79C012656394FE1
:10554000308F278B8E55994F928F818F81E090E01D
:1055500002C0880F991F6A95E2F72091AA06282BAE
:105560002093AA06CF0140E051EE60E070E00E9477
:10557000612ACF91DF911F910F91FF90EF90CF9013
:10558000AF908F900895FC01838D882319F42FEF3D
:105590003FEF0DC00788F08DE02D208131818281A1
:1055A0009381281B390B8481958128233923C901D4
:1055B0000895FC01838D882319F42FEF3FEF11C06C
:1055C000018CF28DE02D2081318182819381281B15
:1055D000390B2095309584819581282339232F5FBD
:1055E0003F4FC9010895FC01838D882361F0A7898D
:1055F000B08D2D913C91119712968D919C9113979E
:105600002817390721F44FEF5FEFCA01089512966A
:105610008D919C9113971696ED91FC911797E80F39
:10562000F91F408112968D919C91139701961496C3
:105630002D913C9115978223932313969C938E93DF
:10564000129750E0E2CFFC01838D882351F0078848
:10565000F08DE02D208131818281938128173907D7
:1056600021F42FEF3FEFC9010895828193810680D5
:10567000F781E02DE80FF91F8081282F30E0F3CF6C
:10568000DC015796ED91FC9158978281938191832B
:1056900080835996ED91FC915A97808191819383F3
:1056A00082830895DC015B968C915B978823A9F136
:1056B0005996ED91FC915A97208131812F5F3F4F90
:1056C00084819581282339235C968C915C9788236B
:1056D00029F08281938128173907F9F0828193811B
:1056E00028173907D9F3808191810680F781E02D51
:1056F000E80FF91F60835996ED91FC915A97318319
:1057000020835296ED91FC915397808156969C91FF
:10571000892B808321E030E002C020E030E0C90125
:105720000895CF93DF93EC011B821A828A819B81BB
:10573000998388831D821C828E819F81009721F02E
:105740000E94C5031F821E82DF91CF9108950F939F
:105750001F938C01DC015296ED91FC9153972081AF
:1057600056968C91569755969C915597892B809576
:105770008223808357968D919C9158970E94912BFC
:10578000F801818D928D0E94912BD8015B961C921D
:105790001F910F9108950F931F93CF93DF938C0167
:1057A000FC0113821282828193819183808341E084
:1057B000A1E0B0E001C04F5FFD01042E02C0EE0F7A
:1057C000FF1F0A94E2F79B0182E06130780710F036
:1057D00020E032E0E217F30770F3C1E0D0E002C04E
:1057E000CC0FDD1F4A95E2F72197F801268137811A
:1057F0002115310541F0848195818C179D0789F031
:10580000C9010E94C503F801D583C483CE01019666
:105810000E941B039C01F8019783868380E0232B61
:1058200009F081E0DF91CF911F910F910895AF9220
:10583000BF92CF92DF92EF92FF920F931F93CF937D
:10584000DF937C015A016B01E901DC015B968C91CD
:105850005B978823F1F02115310539F45796ED91C6
:10586000FC915897C481D58121960115110549F401
:10587000D7015996ED91FC915A97048115810F5FDC
:105880001F4FD701ED91FC910088F189E02DC701F0
:105890000995F7018789908D209711F4C0E8D0E031
:1058A000BE010E94CB2B882381F0D70159968D91A0
:1058B0009C915A970115110511F400E110E0B8010F
:1058C0000E94CB2B882309F04DC0D701ED91FC91AC
:1058D0000088F189E02DC701099567C0D70150966E
:1058E000ED91FC915197B0E0AB16B1EEBB06B0E084
:1058F000CB06B0E0DB0609F454C081E090E0D701AC
:1059000054960C9002C0880F991F0A94E2F7808386
:1059100060E079E08DE390E0A60195010E94EB370D
:105920002150304040405040CA01B90122E030E0EF
:1059300040E050E00E94EB37D7011C96ED91FC91BE
:105940001D9730831E96ED91FC911F972083D70100
:105950005296ED91FC915397808155969C91892B9D
:10596000808323C0D7015996ED91FC915A971382F9
:10597000128282819381918380835796ED91FC916D
:10598000589713821282828193819183808381E070
:105990005B968C931A141B041C041D040CF49ECFFC
:1059A000D6CF108220E130E0C7CFDF91CF911F9199
:1059B0000F91FF90EF90DF90CF90BF90AF90089540
:1059C0002F923F924F925F926F927F928F929F920F
:1059D000AF92BF92CF92DF92EF92FF920F931F93FD
:1059E000DF93CF93CDB7DEB764970FB6F894DEBFE1
:1059F0000FBECDBF3C01688B5A8B498B69011C01DE
:105A0000AE014F5F5F4F5C8B4B8BE989FA89488908
:105A100040FD659140FF6191FA8BE98B662309F4A3
:105A2000D7C3653249F440FD859140FF8191FA8BDF
:105A3000E98B8532B1F40CC06A3051F4D301ED9199
:105A4000FC910190F081E02DC1016DE009956AE0C3
:105A5000D301ED91FC910190F081E02DC1010995F8
:105A6000D4CF982F10E0882499241032B0F49B32C0
:105A700069F09C3228F4903251F0933271F40BC0EB
:105A80009D3239F0903349F4116028C012601460DF
:105A900025C0186023C0106121C017FD2BC0892FBD
:105AA00080538A3078F416FF06C0BAE09B9E902C93
:105AB0001124980E13C0EAE08E9E802C1124880ECB
:105AC00010620CC09E3221F416FD82C3106406C021
:105AD0009C3611F4106802C0983661F4E989FA899D
:105AE000488940FD959140FF9191FA8BE98B99236C
:105AF00009F0BBCF892F8554833020F4812F80613A
:105B0000905E07C0892F8556833008F0E6C1812F4B
:105B10008F7E86FD02C076E0972E6FE3F62EF82288
:105B2000953619F450E4F52A07C0963619F480E842
:105B3000F82A02C091109A94F7FE0BC09BE39915C6
:105B400020F427E05CE3B52E0DC0B92CB39427E018
:105B500009C0A7E0A91520F447E0942E27E001C072
:105B6000292DBB24F6013496FD87EC87D6016D9173
:105B70007D918D919C91AE014F5F5F4F0B2D0E94E7
:105B800043026C010981E02FF0E0FF87EE8700FF00
:105B900005C0FE85F3FD02C01DE209C0F1FE02C092
:105BA0001BE205C0F2FC02C010E001C010E28E85CD
:105BB0009F858C709070892B09F444C0112311F4D7
:105BC00083E001C084E0881510F088240EC0881A94
:105BD000F3FC0BC0D301ED91FC910190F081E02D1D
:105BE000C10160E209958A94A9F7112349F0D30114
:105BF000ED91FC910190F081E02DC101612F09959B
:105C0000BE85B3FF03C00FE013E012C003E113E051
:105C10000FC0E114F10409F06052D301ED91FC9141
:105C20000190F081E02DC10109950F5F1F4F05C064
:105C3000EF2CFF24B0E1EB22FF24F80164916623EE
:105C400041F748C1F7FE13C0BC0CFE85F4FF04C049
:105C50008A81813309F4BA941B141CF0BB24B394D9
:105C60002DC048E04B1550F538E0B32E27C0F6FCA8
:105C700025C0892D90E08C159D054CF05CEFC51674
:105C80005FEFD50624F080E8F82A01C09A949920A5
:105C900049F0E2E0F0E0EC0FFD1FE90DF11D80811D
:105CA0008033A1F3F7FE0AC0B92CB394892D90E09C
:105CB000C816D90614F0992401C09C18F7FC03C03B
:105CC00025E030E009C01C141D041CF021E030E088
:105CD00003C096012F5F3F4F112311F02F5F3F4FFD
:105CE000992029F0892D90E00196280F391F882DE1
:105CF00090E02817390714F0882401C0821A4F2C2D
:105D00005524C20189709070892B59F00CC0D301C1
:105D1000ED91FC910190F081E02DC10160E20995C7
:105D20008A948820A1F7112349F0D301ED91FC91C9
:105D30000190F081E02DC101612F099543FE0BC058
:105D40000CC0D301ED91FC910190F081E02DC101D7
:105D500060E309958A948820A1F7F7FE51C0860177
:105D6000D7FE02C000E010E076010894E11CF11CAF
:105D7000E01AF10AE1E0F0E0EC0FFD1FEE0EFF1E6D
:105D800026014B185108892D90E0AA24BB24A81A9B
:105D9000B90AFFEF0F3F1F0749F4D301ED91FC91C2
:105DA0000190F081E02DC1016EE20995C016D10687
:105DB00034F0401651061CF4F701608101C060E325
:105DC000015010400894E11CF11C0A151B054CF011
:105DD000D301ED91FC910190F081E02DC101099575
:105DE000D8CF0C151D0541F48A81863320F4853304
:105DF00019F4BE85B4FF61E3D301ED91FC9165C058
:105E00006A81613309F00F7ED301ED91FC9101901D
:105E1000F081E02DC10109959920E1F0D301ED91C8
:105E2000FC910190F081E02DC1016EE2099512E034
:105E3000E1E0F0E0EC0FFD1FE10FF11D60811F5F5D
:105E4000D301ED91FC910190F081E02DC101099504
:105E50009A9471F7D301ED91FC910190F081E02DBE
:105E600044FC02C065E601C065E4C1010995D7FCA8
:105E700005C0C114D10441F404FF06C0D094C194FC
:105E8000D108D3946DE201C06BE2D301ED91FC9196
:105E90000190F081E02DC101099560E305C06F5FBD
:105EA000E6EFFFEFCE0EDF1EFAE0CF16D104BCF70F
:105EB000D301ED91FC910190F081E02DC101099594
:105EC000D301ED91FC916C2D605D0190F081E02D8E
:105ED000C1010995CC84DD8478C1933631F09337C4
:105EE00099F0933509F061C023C0F6018081898360
:105EF0005E010894A11CB11C42E050E0C40ED51E06
:105F000021E0E22EF12C12C0D601AD90BC9016FD1E
:105F100003C06FEF7FEF02C0692D70E0E2E0F0E0B8
:105F2000CE0EDF1EC5010E9428047C011F7713C01E
:105F3000D601AD90BC9016FD03C06FEF7FEF02C09D
:105F4000692D70E0E2E0F0E0CE0EDF1EC5010E9498
:105F50001D047C01106813FF0BC023C0D301ED9119
:105F6000FC910190F081E02DC10160E209958A94D5
:105F7000882D90E0E816F90688F313C0F50117FDA7
:105F8000659117FF61915F01D301ED91FC91019043
:105F9000F081E02DC101099581108A940894E108EF
:105FA000F108E114F10451F710C1943611F099365B
:105FB00099F517FF0AC0F601208131814281538192
:105FC00084E090E0C80ED91E0CC0D6018D919C9142
:105FD0009C01442737FD4095542FE2E0F0E0CE0EBF
:105FE000DF1E9FE6F92EF12257FF09C0509540951C
:105FF000309521953F4F4F4F5F4FF0E8FF2ACA0180
:10600000B901AE014F5F5F4F2AE030E00E94E50129
:10601000E82E4B89E41A41C0953721F41F7E2AE00F
:1060200030E01CC0197F9F3661F0903720F498351E
:1060300009F0CEC00FC0903739F0983709F0C8C0CA
:1060400004C028E030E00AC0106114FD146020E1B3
:1060500030E004C014FD166020E132E017FF08C0F4
:10606000D6016D917D918D919C91E4E0F0E008C0A6
:10607000D6018D919C91BC0180E090E0E2E0F0E0DF
:10608000CE0EDF1EAE014F5F5F4F0E94E501E82E8E
:10609000FB89EF1A8FE7F82EF122F6FE0BC04EEFC8
:1060A000F422E91438F4F4FE07C0F2FC05C05FEEF8
:1060B000F52202C01E2D01C0192DF4FE0DC0FE01F7
:1060C000EE0DF11D8081803319F489EEF82208C0AD
:1060D0001F5FF2FE05C003C08F2D867809F01F5F99
:1060E0000F2DF3FC18C0F0FE13C0181510F09E2CF5
:1060F0000FC09E2C980C911A182D0AC0D301ED9157
:10610000FC910190F081E02DC10160E209951F5FD3
:106110001815A0F304C0181510F4811A01C08824C2
:1061200004FF17C0D301ED91FC910190F081E02DA7
:10613000C10160E3099502FF29C0D301ED91FC91F3
:106140000190F081E02D01FD02C068E712C068E512
:1061500010C0802F8678D1F001FF02C06BE201C031
:1061600060E2F7FC6DE2D301ED91FC910190F081CA
:10617000E02DC10109950AC0D301ED91FC91019078
:10618000F081E02DC10160E309959A94E914A0F330
:10619000EA94D301ED91FC91A1E0B0E0AC0FBD1FFA
:1061A000AE0DB11D0190F081E02DC1016C910995FA
:1061B000EE2071F70AC0D301ED91FC910190F081BE
:1061C000E02DC10160E209958A948820A1F71DCCD9
:1061D00064960FB6F894DEBF0FBECDBFCF91DF91AE
:1061E0001F910F91FF90EF90DF90CF90BF90AF90F5
:1061F0009F908F907F906F905F904F903F902F90E7
:106200000895F999FECF72BD61BDF89A80B50895E1
:10621000F999FECF1FBA72BD61BD40BD0FB6F894AB
:10622000FA9AF99A0FBE08950F93FC016115710552
:1062300011F480E011C02183328343835483728739
:1062400061870170000F000F000F8081877F802B16
:1062500082608B7F808381E00F910895CF93DF93DD
:10626000EC010E94E9319B01AC018D819E81AF81DF
:10627000B885281739074A075B0728F4888184FD09
:1062800002C060E00DC089819A81AB81BC81820F20
:10629000931FA41FB51F8D839E83AF83B88761E0D2
:1062A000222757FD2395332744275527922F917096
:1062B0009295907F88818F7E892B8883862FDF91AE
:1062C000CF910895CF93DF93EC01888182FF0FC0B7
:1062D000CE010E942E31882351F0E985FA8530974E
:1062E00009F00995888183FF02C08B7F8883DF9145
:1062F000CF910895CF93DF93EC0189859A85892BFF
:10630000E1F089819A81AB81BC810097A105B1053B
:10631000A1F00E94E93129813A814B815C81260FED
:10632000371F481F591F2D833E834F83588788810D
:1063300084608F7E888381E001C080E0DF91CF910F
:1063400008951F920F920FB60F9211242F933F932F
:106350008F939F93AF93BF938091B2069091B306B2
:10636000A091B406B091B5063091B6060196A11D74
:10637000B11D232F2D5F2D3720F02D570196A11D24
:10638000B11D2093B6068093B2069093B306A093F6
:10639000B406B093B5068091AE069091AF06A09179
:1063A000B006B091B1060196A11DB11D8093AE0655
:1063B0009093AF06A093B006B093B106BF91AF9192
:1063C0009F918F913F912F910F900FBE0F901F9033
:1063D00018958FB7F8942091B2063091B30640918A
:1063E000B4065091B5068FBFB901CA0108959B014B
:1063F000AC017FB7F8948091AE069091AF06A09162
:10640000B006B091B10666B5A89B05C06F3F19F004
:106410000196A11DB11D7FBFBA2FA92F982F8827E4
:10642000860F911DA11DB11D62E0880F991FAA1F43
:10643000BB1F6A95D1F7BC012DC0FFB7F8948091BE
:10644000AE069091AF06A091B006B091B106E6B548
:10645000A89B05C0EF3F19F00196A11DB11DFFBF1C
:10646000BA2FA92F982F88278E0F911DA11DB11D1E
:10647000E2E0880F991FAA1FBB1FEA95D1F7861B80
:10648000970B885E9340C8F2215030404040504006
:1064900068517C4F211531054105510571F608956C
:1064A000019739F0880F991F880F991F029701975C
:1064B000F1F70895789484B5826084BD84B58160D5
:1064C00084BD85B5826085BD85B5816085BDEEE6FC
:1064D000F0E0808181608083E1E8F0E010828081DB
:1064E00082608083808181608083E0E8F0E0808149
:1064F00081608083E1EBF0E0808184608083E0EB69
:10650000F0E0808181608083EAE7F0E08081846050
:1065100080838081826080838081816080838081AC
:10652000806880831092C10008951F920F920FB669
:106530000F9211242F933F934F935F936F937F9309
:106540008F939F93AF93BF93EF93FF938091B70681
:106550009091B806892B29F0E091B706F091B80622
:106560000995FF91EF91BF91AF919F918F917F918D
:106570006F915F914F913F912F910F900FBE0F90B0
:106580001F9018951F920F920FB60F9211242F9300
:106590003F934F935F936F937F938F939F93AF93AB
:1065A000BF93EF93FF938091B9069091BA06892B20
:1065B00029F0E091B906F091BA060995FF91EF91A3
:1065C000BF91AF919F918F917F916F915F914F910B
:1065D0003F912F910F900FBE0F901F901895CF9362
:1065E000DF93482F50E0CA01875B9C4FFC01349138
:1065F0004B5C5C4FFA018491882369F190E0880F2D
:10660000991FFC01E95EFC4FA591B491FC01EF5D7F
:10661000FC4FC591D491662351F42FB7F8948C9117
:10662000932F909589238C93888189230BC06230A6
:1066300061F42FB7F8948C91932F909589238C93C4
:106640008881832B88832FBF06C09FB7F8948C91D5
:10665000832B8C939FBFDF91CF910895482F50E0FB
:10666000CA01835A9C4FFC012491CA01875B9C4F4D
:10667000FC0194914B5C5C4FFA013491332309F493
:1066800040C0222351F1233071F0243028F421300E
:10669000A1F0223011F514C02630B1F02730C1F03E
:1066A0002430D9F404C0809180008F7703C080919A
:1066B00080008F7D8093800010C084B58F7702C0EA
:1066C00084B58F7D84BD09C08091B0008F7703C0F1
:1066D0008091B0008F7D8093B000E32FF0E0EE0F4B
:1066E000FF1FEF5DFC4FA591B4912FB7F89466237F
:1066F00021F48C919095892302C08C91892B8C93E5
:106700002FBF08958093BC020895982F8E3008F013
:106710009E5097708091BC028295880F880F807C74
:10672000892B80937C0080917A00806480937A002A
:1067300080917A0086FDFCCF20917800409179000D
:10674000942F80E030E0282B392BC9010895CF9297
:10675000DF92EF92FF920F931F93CF93DF937C0111
:106760006B018A01C0E0D0E00FC0D6016D916D01D0
:10677000D701ED91FC910190F081E02DC7010995C1
:10678000C80FD91F015010400115110571F7CE0136
:10679000DF91CF911F910F91FF90EF90DF90CF90FD
:1067A0000895CF93DF930E945A320E940228C0E0DE
:1067B000D0E00E94302A2097E1F30E940000F9CF38
:1067C0005058BB27AA270ED041C201D230F006D2C2
:1067D00020F031F49F3F11F41EF4C0C10EF4E09597
:1067E000E7FBB6C1E92F54D280F3BA1762077307EB
:1067F0008407950718F071F49EF56CC20EF4E095CD
:106800000B2EBA2FA02D0B01B90190010C01CA016A
:10681000A0011124FF27591B99F0593F50F4503E15
:1068200068F11A16F040A22F232F342F4427585F07
:10683000F3CF469537952795A795F0405395C9F71F
:106840007EF41F16BA0B620B730B840BBAF09150D7
:10685000A1F0FF0FBB1F661F771F881FC2F70EC076
:10686000BA0F621F731F841F48F487957795679549
:10687000B795F7959E3F08F0B3CF9395880F08F032
:106880009927EE0F979587950895A1D158F080E844
:1068900091E009F49EEFA2D128F040E851E059F4CC
:1068A0005EEF09C05BC116C2E92FE078F1D168F351
:1068B000092E052AC1F3261737074807590738F06C
:1068C0000E2E07F8E02569F0E025E0640AC0EF63CA
:1068D00007F8009407FADB01B9019D01DC01CA0148
:1068E000AD01EF934AD0B2D10AD05F91552331F078
:1068F0002BED3FE049E450FD49EC63CF0895DF9371
:10690000DD27B92FBF7740E85FE316161706480763
:106910005B0710F4D92FE9D19F938F937F936F93E7
:10692000BCD2E8E6F0E01DD191D12F913F914F917B
:106930005F91EED1DD2349F09058A2EA2AED3FE0C5
:1069400049EC5FE3D0785D274DDFDF917FC1DCD07C
:1069500008F481E008954AD1E39589C10CD076C14D
:106960003DD140F034D130F021F45F3F19F0F0C058
:106970005111B1C1F3C08CD198F39923C9F35523B8
:10698000B1F3951B550BBB27AA2762177307840722
:1069900038F09F5F5F4F220F331F441FAA1FA9F3D8
:1069A00033D00E2E3AF0E0E830D091505040E695CA
:1069B000001CCAF729D0FE2F27D0660F771F881F2B
:1069C000BB1F261737074807AB07B0E809F0BB0B1A
:1069D000802DBF01FF2793585F4F2AF09E3F51053E
:1069E00068F0B6C078C15F3FECF3983EDCF3869563
:1069F00077956795B795F7959F5FC9F7880F911DB4
:106A00009695879597F90895E1E0660F771F881F9F
:106A1000BB1F621773078407BA0720F0621B730B52
:106A2000840BBA0BEE1F88F7E095089504D06894A4
:106A3000B11151C1089534D188F09F5790F0B92F0A
:106A40009927B751A0F0D1F0660F771F881F991FC3
:106A50001AF0BA95C9F712C0B13081F03BD1B1E05C
:106A6000089538C1672F782F8827B85F39F0B93F6C
:106A7000CCF3869577956795B395D9F73EF49095C5
:106A80008095709561957F4F8F4F9F4F0895E89443
:106A900009C097FB3EF490958095709561957F4F66
:106AA0008F4F9F4F9923A9F0F92F96E9BB27939514
:106AB000F695879577956795B795F111F8CFFAF424
:106AC000BB0F11F460FF1BC06F5F7F4F8F4F9F4F55
:106AD00016C0882311F096E911C0772321F09EE8B3
:106AE000872F762F05C0662371F096E8862F70E019
:106AF00060E02AF09A95660F771F881FDAF7880FF3
:106B00009695879597F90895990F0008550FAA0B48
:106B1000E0E8FEEF16161706E807F907C0F01216B0
:106B20001306E407F50798F0621B730B840B950BB3
:106B300039F40A2661F0232B242B252B21F4089508
:106B40000A2609F4A140A6958FEF811D811D0895A5
:106B500097F99F6780E870E060E008959FEF80EC10
:106B60000895DF93CF931F930F93FF92EF92DF92DD
:106B70007B018C01689405C0DA2EEF01C9D0FE01BB
:106B8000E894A5912591359145915591AEF3EF018A
:106B900029DEFE019701A801DA9479F7DF90EF90E2
:106BA000FF900F911F91CF91DF9108959F938F9345
:106BB0007F936F93FF93EF939B01AC019DD0EF9177
:106BC000FF91CFDF2F913F914F915F9195C00024AE
:106BD0000A941616170618060906089500240A9442
:106BE00012161306140605060895B8CF59D0E8F317
:106BF000E894EFEFBB273FE048EC5FE76B3D73079E
:106C00008407950708F1FF279F57B25A6A4D7F40C6
:106C1000894CF04032F4BE556542704F8643FF4FB9
:106C20000894EE1F915030F0BB0F661F771F881F2E
:106C3000FF1FEBCF9EE7882332F0BB0F661F771F45
:106C4000881F9A95C1F79395E09565C1092E039425
:106C5000000C11F4882352F0BB0F40F4BF2B11F449
:106C600060FF04C06F5F7F4F8F4F9F4F0895EF937A
:106C7000E0FF06C0A2EA2AED3FE049EC5FEBB2DD9F
:106C8000E5DF0F90039401FC9058E5E9F0E08ECF2A
:106C900057FD9058440F551F59F05F3F71F04795CD
:106CA000880F97FB991F61F09F3F79F087950895B2
:106CB000121613061406551FF2CF4695F1DF08C0D1
:106CC000161617061806991FF1CF869571056105EE
:106CD00008940895E894BB2766277727CB0197F996
:106CE000089512DF08F48FEF08959B01AC0160E076
:106CF00070E080E89FE332CE0BD0A8CF68DF28F0A9
:106D00006DDF18F0952309F023CF28CF1124E3CFAE
:106D1000BFDFA0F3959FD1F3950F50E0551F629F01
:106D2000F001729FBB27F00DB11D639FAA27F00DE4
:106D3000B11DAA1F649F6627B00DA11D661F829F0B
:106D40002227B00DA11D621F739FB00DA11D621FF0
:106D5000839FA00D611D221F749F3327A00D611D0D
:106D6000231F849F600D211D822F762F6A2F1124EF
:106D70009F5750408AF0E1F088234AF0EE0FFF1F42
:106D8000BB1F661F771F881F91505040A9F79E3F79
:106D9000510570F0DDCE9FCF5F3FECF3983EDCF302
:106DA000869577956795B795F795E7959F5FC1F7B6
:106DB000FE2B880F911D9695879597F9089570DFA2
:106DC000E0F09E37D8F09639B8F49E3848F4672F33
:106DD000782F8827985FF9CF869577956795939553
:106DE0009539D0F3B62FB1706B0F711D811D20F452
:106DF000879577956795939573C08DC06CCF11F487
:106E00000EF4ACCE88C04CDFD0F39923D9F3CEF387
:106E10009F57550B87FF8FD056959795B0E020F47C
:106E2000660F771F881FBB1F1F930F9300249001CD
:106E3000A0018001F001A0E80E0F1F1F0A1E511DC6
:106E4000601B710B8009B50B48F4600F711F801D2A
:106E5000B51F0E1B1F0B0A0A510907C02E0F3F1F3B
:106E60004A1F0E0F1F1F0A1E511D660F771F881F16
:106E7000BB1FA695F795E795F8F6061717070806BE
:106E80005B07211D311D411D0F911F91B901842FF9
:106E90009158880F9695879508959B01AC012CCF4A
:106EA000DF93D92FA3DEE695D7952AED3FE049E49D
:106EB0005FE3B33A6207730784079507D7952AF013
:106EC000A2EA49EC90688EDCC1DEE3EBF0E06EDE16
:106ED000DD0F0BF00ADFDD0F0BF49058DF91089502
:106EE000882371F4772321F09850872B762F07C0E1
:106EF000662311F499270DC09051862B70E060E055
:106F00002AF09A95660F771F881FDAF7880F9695F3
:106F1000879597F908959F3F49F0915028F48695F9
:106F200077956795B7959F5F80389F4F880F9695A7
:106F3000879597F9089591505040660F771F881FE5
:106F4000D2F70895AA1BBB1B51E107C0AA1FBB1FA4
:106F5000A617B70710F0A61BB70B881F991F5A95E5
:106F6000A9F780959095BC01CD01089597FB092E56
:106F700007260AD077FD04D0E5DF06D000201AF4FA
:106F8000709561957F4F0895F6F7909581959F4F85
:106F90000895A1E21A2EAA1BBB1BFD010DC0AA1F5A
:106FA000BB1FEE1FFF1FA217B307E407F50720F072
:106FB000A21BB30BE40BF50B661F771F881F991FED
:106FC0001A9469F760957095809590959B01AC0136
:106FD000BD01CF01089597FB092E05260ED057FD60
:106FE00004D0D7DF0AD0001C38F450954095309576
:106FF00021953F4F4F4F5F4F0895F6F7909580953D
:10700000709561957F4F8F4F9F4F0895EE0FFF1F33
:0C7010000590F491E02D0994F894FFCF56
:10701C0025630025632563002563253269256325D7
:10702C003032697C2563253269256325303269004D
:10703C0025632532692563253032690025352E30CC
:10704C0066256300256325312E356625630025638F
:10705C00253569256300256325352E3266256300A9
:10706C006D616E007374310073743200737433008D
:10707C0073743400737435007374360070682000B8
:10708C00636C200076722000686C20006170200018
:10709C00727462006C616E0070702000706F690019
:1070AC006163200000617420002563257300256353
:1070BC0025332E306925630025346925632563004B
:1070CC00256325336925630025737C25632573258A
:1070DC00630020C0C0C0C0C0C7C0C0C0C0C02000BA
:1070EC0025342E3066256300256325332E30662526
:1070FC006300256325352E30662563002563253115
:10710C00312E36667C25632531312E36660025639B
:10711C002532690025332E3166256300202020207E
:10712C002020202020202020002020646973617200
:10713C006D6564202000206E6F2074656C20636F79
:10714C006D2000206E6F20677073206669782000B8
:10715C00202062617474206C6F772020006261744F
:10716C0074207761726E696E670062617474637209
:10717C0069746963616C0020626174742065727259
:10718C006F722000202072737369206C6F7720203F
:10719C00006D6167207761726E696E67006D616763
:1071AC0020637269746963616C00206D61672020D3
:1071BC006572726F7220002573002000BF060000FC
:1071CC00E803E803E803E8039DFF01640100000005
:1071DC00007B05A73379047C047F0482043C2A00DD
:1071EC00070E091C1B1215383F363124232A2D702B
:1071FC00777E796C6B6265484F464154535A5DE01B
:10720C00E7EEE9FCFBF2F5D8DFD6D1C4C3CACD90CA
:10721C00979E998C8B8285A8AFA6A1B4B3BABDC733
:10722C00C0C9CEDBDCD5D2FFF8F1F6E3E4EDEAB76A
:10723C00B0B9BEABACA5A28F88818693949D9A27DA
:10724C0020292E3B3C35321F18111603040D0A570A
:10725C0050595E4B4C45426F68616673747D7A89F8
:10726C008E878095929B9CB1B6BFB8ADAAA3A4F9AA
:10727C00FEF7F0E5E2EBECC1C6CFC8DDDAD3D4699A
:10728C006E676075727B7C51565F584D4A4344194A
:10729C001E171005020B0C21262F283D3A33344EB5
:1072AC0049404752555C5B7671787F6A6D64633EEA
:1072BC0039303722252C2B0601080F1A1D1413AE5A
:1072CC00A9A0A7B2B5BCBB9691989F8A8D8483DE8A
:1072DC00D9D0D7C2C5CCCBE6E1E8EFFAFDF4F3C2C6
:1072EC00C0C0C1C0C0C1C0C0C4C0C0C1C0C0C1C08A
:1072FC00C0C3C0C0C1C0C0C1C0C0C5C0C0C1C0C077
:10730C00C1C0C000000000522BA733C32AF32A23AC
:0C731C002B402BD92A612AA72B172C002C
:00000001FF
